:020000041100E9
:103000000023F7B52E4D2F4C280063616374022610
:1030100001F076F94021FE22217428002A4B009607
:1030200001F0C0F900283AD1217CFF222800274B6B
:10303000009601F0B7F9002831D1254BA2899A42B8
:103040002AD1E389234A934211D1234B6361234B55
:103050002268002A07D1002B05D019002200C1C91F
:10306000C1C21B7B6374280001F088F9F7BD1C4ABC
:10307000934201D00023EBE71A4B1B4A1B68934293
:1030800006D9C02304222800217C9B0001F000FA0D
:10309000164B6361164BDBE700232374EAE7CC236E
:1030A0003821AC2228009B01217401F0F1F900289D
:1030B000F2D1104B6361104BE381104BC8E7C0465F
:1030C000D441FF1FA061FF1FAC61FF1FAE61FF1F56
:1030D00059590000830500003141001180BD0011E5
:1030E00082150000C461FF1F87130000E541001135
:1030F00090BD00117D410011AAAAFFFF70BD001113
:10310000F7B5164B0192C318021D002000938823C7
:103110005B05D3181B685C1C1AD09CB2402C18D8D5
:103120008D781E0CAC466746CD782D023D43AE42ED
:1031300006D1019800280ED110000C70240A4C70A2
:1031400003249BB20733A343D218009B9A42DED3D9
:10315000FEBD4432F9E71000FAE7C046FC0F00005C
:10316000802213B503000324019189B25201073173
:103170009B18A14304305A1A88235B05C3181B68A7
:10318000591C03D190429241104016BD99B240297A
:1031900007D80B000733A343C0189042ECD300209C
:1031A000F3E74430F9E7134B134A1B68126810B574
:1031B000FA24934201D81A00F824104BE4021B6849
:1031C0009A4210D813000E4A12689A420ED3013365
:1031D00007D1F823DB029C4203D10A49054808F0D5
:1031E00023FB200010BDFC24E402ECE7FE24E402F3
:1031F000F7E7C04600C0071100D0071100E0071133
:1032000000F00711FFFFFF7FF0B59BB015000490A1
:103210000391402A00D9A0E006AB59801A80FFF73D
:10322000C2FF0400042816D9002206A9FFF768FF90
:10323000052810D906AB1B88AB420CD1002D07D056
:10324000514B2A000499C01808F0FEFC002802D156
:1032500001201BB0F0BD06AB1D8020000699FFF7D2
:103260007FFF041E7BD1069B0793FFF79CFF802303
:103270005B01C618802307001B039E4201D3F8267A
:10328000F60288235B05F31801931B68013302D013
:10329000019808F051FB3D49019808F0C5FA3B1D23
:1032A0000293331D05938822029B52059B181B68CD
:1032B00008935A1C3CD044219AB20091402A04D869
:1032C0000320D11D814389B2009103991B0C8B42CD
:1032D00024D0402A22D80122300008A9FFF710FF8D
:1032E000021E1BD1380008A9FFF70AFF04000428BA
:1032F00031D9009A059B9B1880225201B218934243
:1033000040D288235B05C118009A09A808F0F4FB95
:103310001D4B009A09A9F01808F006FC009A029BC0
:103320009446634402931A4B029AFB189A42BAD30A
:1033300088235B05FC1821680198013908F074FAAC
:10334000200008F0F9FA039A07AB5A803000079979
:10335000FFF706FF0400002C03D1002079E70428C2
:10336000FBD988235B05E018069908F05DFA032372
:10337000EA1C9A4300D16BE7034B0499E01808F06C
:10338000D3FB65E70424ECE704000011FFFFFF7F97
:10339000F80F0000F7B505001400402A21D80027D7
:1033A00001AE71803780FFF7FEFE042816D93A007F
:1033B0003100FFF7A5FE042810D93688BC420BD097
:1033C000BD4209D0221CB44200D9321C064B92B235
:1033D000C118280008F090FB30B2FEBDC04300B217
:1033E000FBE703204042F8E70400001137B5042250
:1033F00004000D0001A81649FFF7CCFF02000428C5
:103400000BD1019BA34208D3AB4204D0104901A8C1
:103410000195FFF7F9FE01203EBD0E4C2368200008
:10342000019308F089FA019920000139019108F00F
:10343000FBF980235B01E418074B9C42EED1042288
:10344000034901A80195FFF7DFFE0020E4E7C0462D
:103450005555000000C007110000081130B589B0B3
:1034600008F08AFA10226946254808F0B5F9254B7C
:10347000009A9A420ED1019B029A0F2B33D8002159
:1034800001240698013B08D2002900D00292029B39
:10349000013331D10023029325E0551CF2D1020003
:1034A0002100EFE710341022200004A908F094F95D
:1034B000029B013301D1069B0293882304995B058B
:1034C000C918059B06981A03120B049105928142B4
:1034D00003D02B4201D108F00FFB019B013B01936C
:1034E000019B002BDED1029B002B03D00493049898
:1034F0004168084709B030BDE025014C2D03EFE7D6
:1035000000000111504859368022F8B5964C974B6F
:10351000D200002120001C6008F046FB2300944AE2
:1035200088331A60934B1A786A23002A00D011332B
:10353000E3620A232365904B37221B780820A3639C
:103540008E4B2118E361102323628D4B3B25636171
:10355000C823DB00A36123008C331A602823013ABF
:10356000E26320646364CA67043A211DCA672100CC
:10357000BC310D602100C03108602100C4310B60F6
:1035800021000635CC310D602100083DC8310D60A9
:103590002100D0310A602200D43210602200D832DB
:1035A000136022000227E032210017604222DC3142
:1035B0000A6021001B3DE4310D602100E831086004
:1035C0002100EC310B6023000521F4331960230046
:1035D000F0331A602300183290331A6023009433BA
:1035E000186023001E3A98331A60AF23DB00236073
:1035F000644BFA262363644B644DE360644BF03103
:10360000A3642300FF31FC33B600A16021611E607A
:10361000A5627325E5656D3D6565A56596255D4AE1
:10362000AD00E264666258606766A56600270925FA
:10363000A767E566584F594D606720002567E26728
:103640003A6015279C30676007001A203860200018
:10365000A0300700212038602000A83007004C4827
:1036600038602000F830066026006427A4363760F2
:1036700026005F3FAC3637602600033FB036376028
:103680002600C637B436376026000027B8363760C4
:1036900038269E60424E96205E64424E5A66DE6137
:1036A000414E9A645E62F53EFF3E9E621E269A6718
:1036B000354A8000DE661F675F67DD651D6618623C
:1036C000DA67BE23394A5B00E250394BD8382350C1
:1036D00004302250C4225200A350C623E4205B00D1
:1036E000E1500433334AE1503349344BD16034491B
:1036F000800019503349E938FF38195032490430F5
:10370000195032493248D16132491163324951630B
:103710001900F4310860CE20304940001160304972
:10372000195019002F48F83108602F49D1658221BE
:103730002E4A89005A501A002D490832D1671A00C2
:103740002C49B432116088212B4A89005A501A0042
:103750002A49883211602A4ADA6408F04DF80120BB
:1037600008F0D2F9F8BDC0460004FF1F4464FF1FF3
:10377000106FFF1F1044FF1F4A0AFF1F3A07000087
:1037800080C3C9019A020000DC0500006A1800002D
:1037900050C3000088130000F009FF1F204E0000F6
:1037A0006509FF1F68100000C409000040420F00B7
:1037B00010270000FC00FF1F751CFF1F0000FF1FEB
:1037C000C92CFF1F5130FF1FE92EFF1F3520FF1F9F
:1037D0002527FF1F5120FF1FFD21FF1FC11FFF1FB6
:1037E0004929FF1F312AFF1F8D19FF1F5528FF1F71
:1037F0007925FF1F8525FF1FC11EFF1F791FFF1F92
:10380000391EFF1F0223F0B50124624D624E2B705A
:10381000624B91B01C70624F039333680021082003
:10382000FB7006F00DFE082006F004FD0023984210
:1038300005D0FA78552A02D0332A00D09DE03360B3
:10384000042006F077FF08F007F8FFF75DFE08F0A8
:1038500063F91F2201240021524B10AE1A70524B03
:103860001C70524B1970524B19689143163A0A4317
:103870001A60602219689143403A0A431A6008F0BE
:10388000ABF907F031FF4B4B9847C120FF214A4B62
:1038900080001A588A431A50C522920098588843CB
:1038A000BF39014399509858444908408021C901C3
:1038B0000143802099509958C0050902090A014323
:1038C000995080213E48490107F076FF03232200EA
:1038D0003C49019400933C4807F0DEFE2C223B4912
:1038E00005A808F009F905AC61782078023406F0E3
:1038F000C1FCA642F8D1364C0020012106F0CEFDD5
:103900002268344B03201A40A023DB0213432360B8
:10391000802322689B041343236022682E4B1A40A5
:1039200080239B03134323602C4A2D4B934200D8E2
:10393000012008F099F908F017F980232268DB04C8
:1039400013432360287808F02FF8039B1878C0B23F
:1039500008F052F808F0F0F82249042008F044F882
:1039600006F0B4FE00F040F800F0E8FD00F090FE34
:1039700000F00CFA002011B0F0BD00932100194AAC
:10398000042007F0C1FF8023DB059C62FFF766FD82
:1039900056E7C0464A0AFF1F34F000401044FF1F9C
:1039A000D061FF1F480AFF1F490AFF1F680AFF1F57
:1039B000BCF00040E1A2000000E100E0FF00FFFFDA
:1039C0001444FF1F9856FF1F1454FF1F98BC00118A
:1039D00014F00040FF7FF8FFFFFF9FFF0080FF1FF4
:1039E000106FFF1F3B000108002210B511001120CD
:1039F00007F06AFF10BD0000F8B500230926374F15
:103A0000374C3B62E3681120B343E36008F09CF855
:103A1000112007F0A9FE112008F006F840232268C3
:103A200080251343236080236268DB0213436360B5
:103A3000A3682C4A2B43A360A36802211340A36010
:103A40008023A2689B0113431022A360236C0720EC
:103A500093432364236C0F3A1343236480235B0056
:103A60003B62226B204B1A402263626B1A406263F6
:103A7000A26B1A40A263E26B1340E363E3681B4A44
:103A80001340E36006F0F6FB0121072006F006FD77
:103A9000174B11205A6C15435D6407F005FFFD219B
:103AA000144B154A89005A508023C720626B5B0370
:103AB00013436363E36880003343E3600F4B104AB2
:103AC00019581140802212020A431A50802292058E
:103AD0001A6008220B4B5A63F8BDC04600F0004044
:103AE0003CF00040FFFFDFFFEFFFEFFFFFFF7FFF36
:103AF000003800400000FF1F5118FF1F00E100E0E8
:103B0000FF00FFFF0000054070B5284C238C002B00
:103B100023D0228A002A21D1DA0023826382A38261
:103B2000E38223836383A383E38322606260A260D2
:103B3000E2601F4D1F4A6420EB8093420AD8FA22AC
:103B40000020D200934205D91B4A0A21981807F099
:103B500073FDC0B200232872238470BD0720E11CCE
:103B6000CA7F01320240CA7705D10325201DC17FDB
:103B700001312940C17708325200A35200232100AD
:103B80001A00088A01321B180231082AF9D1221DB5
:103B9000D27F9200A350626823689B18A2689B188A
:103BA000E2689B185B099BB2C3E7C0461061FF1F28
:103BB000B861FF1FB70B000030F8FFFF30B503A856
:103BC00004880B20002C0ED14968074D08784978ED
:103BD000090201430A20A94205D1012120001980D0
:103BE000024B1B7A137030BD192A0000B861FF1F09
:103BF000F7B5150008AA16884A680F4F147852784E
:103C0000120222430A24BA4214D10122DBB20192E9
:103C100000962A0007F0AAFC041E0BD1074B1B6874
:103C2000002B07D068782A780002104342425041A6
:103C3000013098472000FEBD022900003C61FF1FB3
:103C400030B5012503790400BFB02B4211D00A49D9
:103C5000408806F0F7FF28420BD0084B01A95B8D86
:103C60004D800B80064B00221B7A60880B7104F09C
:103C7000C9F83FB030BDC0463461FF1F4840FF1F48
:103C8000B861FF1F10B50549054806F091FF0421F2
:103C9000044A054806F04EFF10BDC0463461FF1FC0
:103CA000FFFF0000C4BC00114840FF1F10B50248D0
:103CB00004F02AFF10BDC046413C001101230370EF
:103CC0000B4B1A7A4270022282709A78C270DA78AC
:103CD0000271032242711A7982715A79C2710C22DF
:103CE00002729A794272DB7983720B207047C04668
:103CF000B861FF1F022310B50370013B4370053309
:103D0000837010330371443B43712A33837144330E
:103D1000C37100230372064B04001B8843720A30F0
:103D2000FFF7CCFF831D0A30C0B2E37010BDC04660
:103D3000B861FF1F10B5142007F0F6FC124B1422D7
:103D40000021186007F030FF002007F0F5FC01208B
:103D500007F072FE022007F0AFFD032004F078F9AF
:103D6000042006F08DF9052003F0B6FB062004F0D0
:103D700083F8072001F06CFA082006F0BBFE09204A
:103D800001F038F810BDC0464061FF1F07F06CFE1F
:103D9000012007F091FE07F087FE0000094B10B5E7
:103DA0000400984205D0012904D12000064906F0FC
:103DB000FFFE10BD0229FCD1013904F063FE00288A
:103DC000F3D0F6E7FEFF00006661FF1F70B50D7AC5
:103DD000100004AA2C00168810221440154220D18D
:103DE000002E20D10A78022A18D14A685178157815
:103DF0000E4A09022943914205D00D4A914209D049
:103E00001C800A2404E014220A491A8007F074FE78
:103E1000200070BD0C2208491A80F7E71C8001249D
:103E2000F6E70824F4E70B24F2E7C046F3FF0000AE
:103E3000F4FF00009C42FF1FACBD001110B5040050
:103E40000749084806F0B4FE074804F09DFD00202D
:103E5000E40704D50721054A054806F06BFE10BDAE
:103E60006661FF1FFFFF00009D3D001108BD0011AE
:103E70008C40FF1F00B50C4BBFB01A780B4902A84D
:103E800000F0C0FC6B4680B2D880002809D06A469A
:103E9000074B01A91B889380064B0022188803F06A
:103EA000B1FF3FB000BDC0464461FF1F4561FF1F29
:103EB000E640FF1FF041FF1F00B50C4BBFB01A7862
:103EC0000B4902A801F0E4FE6B4680B2D8800028BE
:103ED00009D06A46074B01A95B8D9380064B0022EF
:103EE000188803F08FFF3FB000BDC0466E61FF1F12
:103EF0006F61FF1F8C40FF1FF041FF1FF7B50E00E1
:103F0000377A1C0008AB11003D001A8820231D40A1
:103F10001F423CD13378022B3BD173681F785B780A
:103F20001B023B431E4FBB4208D01E4FBB4214D066
:103F30001D4DAB4221D00A252800FEBD002A2AD102
:103F4000142C2AD82200F06807F0D6FD174B1C70FD
:103F5000012CF1D9FFF7B0FFEEE7002A1BD1202C8E
:103F60001BD82200F06807F0C7FD114B04211C701C
:103F7000104B187807F078FCDEE7E3B201240092DA
:103F800001940A00310007F0F1FA0500D4E7082592
:103F9000D2E70125D0E70B25CEE70D25CCE7C046BB
:103FA000F3FF0000F4FF0000022900006E61FF1F14
:103FB0004461FF1FF061FF1F332310B5040003703D
:103FC0000A220749013007F097FD064B0F201B68B6
:103FD0001A0AE37222731A0C1B0E6273A37310BDCC
:103FE000B861FF1FE061FF1F30B5012503790400B0
:103FF000BFB02B4213D00B49408806F023FE284265
:104000000DD06A46084B02A81B889380FFF7D4FFA7
:104010006B46D8800022608801A903F0F3FE3FB010
:1040200030BDC0466661FF1FE640FF1F10B5024865
:1040300004F06AFD10BDC046E93F001170B51600DE
:1040400004AA148805AA15784A68507811780002E5
:104050002A4A0843801805284BD807F0CDFD0313E2
:104060001E29343F0720032C0BD80422121BAA421E
:1040700000D92A0022491A803000091907F03CFDB6
:10408000002070BD0720112CFBD81222121BAA425F
:1040900000D92A001B491A80EEE707200E2CF0D821
:1040A0000F22121BAA4200D92A0017491A80E3E7FF
:1040B0000720032CE5D80422121BAA4200D92A00AB
:1040C00012491A80D8E70720032CDAD80422121BE1
:1040D000AA4200D92A000E491A80CDE70720032CF6
:1040E000CFD80422121BAA4200D92A0009491A80FB
:1040F000C2E700220A201A80C3E7C046DCD5FFFFD2
:1041000053BD00118C61FF1F43BD00113EBD001166
:1041100039BD001134BD001110B50D21024A03480C
:1041200006F008FD10BDC04628BD0011FC40FF1F71
:1041300013B5104C0423217C01AA00F061F900287A
:1041400015D16B469A88236852BA92B2534322899A
:1041500009491B0C9B184B806B46DA88636852BA7E
:1041600092B2534362891B0C9B188B8016BD0120B1
:10417000FCE7C046A061FF1FB861FF1F37B5174CB1
:1041800007236A46217C00F03BF9002824D16B46C6
:104190001B787F2B20D86B46DD78F0232A041B0385
:1041A0001A406B469B880E495BBA9BB21A43236840
:1041B0002D09534322891B0C9B184B806B465A7860
:1041C0009B7812031B011A4363682A435343628995
:1041D0001B0C9B188B803EBD0120FCE7A061FF1FDC
:1041E000B861FF1F7FB50226154C0022217C03AB6E
:1041F0000096050000F0D6F8002802D0012004B097
:1042000070BD0E23217C0122280000966B4400F033
:10421000C9F80028F2D16B469A892368D2BA534371
:10422000228908491B149B184B806B46DA89636806
:1042300052BA92B2534362891B0C9B188B80DEE703
:10424000A061FF1FB861FF1F70B5114C237C002BCC
:104250000FD0382B0ED10F4D280000F051F8CC2391
:10426000AC222800217C9B0100F012F9280000F00C
:1042700085F870BD084BE2899A42FAD1054D2800B5
:1042800000F03EF800222800217C00F0E3F8EDE782
:10429000A061FF1FD441FF1F8305000070B5144CBF
:1042A000237C002B1FD06369002B1CD0114D2800EC
:1042B00000F026F86369280098470400280000F001
:1042C0005DF8002C10D10C4B0422995E002905DA10
:1042D0009C801A8801321A80200070BD074A9142E2
:1042E000F7DD9A80F5E70124FEF78AFEF4E7C04681
:1042F000A061FF1FD441FF1FB861FF1F0F270000FF
:1043000070B5C17905000C00631E9C411A4BE40294
:10431000E41849000460C9B2007906F0F5F8E979BB
:10432000687949000131C9B206F0EEF8E879093040
:10433000C0B207F079FB0023E36661332360AA79FA
:104340005B3B002A0ED022689A43023B1343236052
:104350000A23E3610733236200232363A36301334A
:10436000E36370BD22689A4302231343236046230C
:1043700063610633A361EFE70050004070B500258C
:1043800004000368DD66C0790930C0B207F0DCFBC9
:104390002900207906F054F82900607906F050F8D9
:1043A00070BD0000F8B51E0006AB1D780023046840
:1043B0001700E366616007F0DFFA01238022E366FD
:1043C0002B0027615200013B08D207F08DFB08202B
:1043D0000A4A1168002D03D12800F8BD2261F2E7D6
:1043E000236F034203D02369013D33700136136804
:1043F0005B1A032BEED90125EEE7C0466008FF1FCC
:1044000070B51C00002305681600EB66696007F0B4
:10441000B3FA01238022EB6623005200013B08D24D
:1044200007F062FB08200A4A1168002C03D1200023
:1044300070BD2A61F2E72B6F034203D02B69013C68
:104440003370013613685B1A032BEED90124EEE7B3
:104450006008FF1F002370B504681500E366616003
:1044600007F08AFA0123E366256107F03DFB80200F
:10447000064A80001168636B034205D113685B1A1A
:10448000032BF8D9012070BD0020FCE76008FF1F56
:1044900070B51D00002304681600E366616007F034
:1044A0006BFA0123E36626610F33626B1A42FCD07C
:1044B0002B0A23611023626B1A42FCD0EDB22561F6
:1044C00007F012FB8020074A80001168636B0342EB
:1044D00005D113685B1A032BF8D9012070BD0020A9
:1044E000FCE7C0466008FF1F70B51E00002305688A
:1044F0001400EB66696007F03FFA0123A619EB662A
:104500000F33B4420ED107F0EFFA80200A4A800040
:1045100011686B6B03420CD113685B1A032BF8D93B
:10452000012070BD21782961696B1942FCD00134EA
:10453000E7E70020F5E7C0466008FF1F10B5084C0C
:10454000E368002B08D18022064B52021B689B189F
:104550006360054B1B68236007F01EF9A06010BD67
:10456000E061FF1FC8F00040CCF0004070B5184A71
:10457000936A916A9942FBD116498A689A421FD37D
:104580009A1A8B60144B0126186893B2D202D20E8D
:104590004343424300204C681B0A1B1912029B181C
:1045A0000E4C0A684B60551CA3420CD8002801D061
:1045B0004B600A600A4A136008680A4B186070BDB5
:1045C000581E821ADDE7084A30009B182A00EAE7E5
:1045D00000F00040E061FF1F140AFF1F40420F007F
:1045E000C8F00040CCF00040C0BDF0FF70B51F4CDB
:1045F00023793F2B01D93F2323711D4B22791A7058
:104600001878C0B207F020F818231A491A4A0B800C
:104610001A4913800B805380A379194980200B809D
:104620000C21938001334B43164D191C000183422A
:1046300000D9011C2980D1806379002B11D101336D
:104640006371237A012B01D8022323726279237AC2
:104650000D4853430A21584306F0EEFF0B4D2860E6
:1046600070BDA02BEDD9A023EAE7C046D461FF1F9F
:10467000480AFF1FEE41FF1FBC43FF1FEC41FF1F15
:10468000EA41FF1FE841FF1F71020000C461FF1FE4
:10469000F8B519210020FEF7A9FE114C011E114D9D
:1046A00009D10C22104BC1CBC1C4280007F07CFA01
:1046B000FFF79CFFF8BD0C2220000C49FEF76AFEB4
:1046C0000C2802D0084B43CB43C40C2228000849D5
:1046D000FEF760FE0C28EBD00C220021E5E7C04677
:1046E000D461FF1FA061FF1FA0BD0011FC0C0000E2
:1046F000F50C0000F0B51D4C8022A5440400882074
:1047000069465201400507F037F8902212016A44C9
:104710001300200032C832C316C816C38023144CBD
:10472000144FA6689B033343A3603B6007F0B4F9C2
:104730008823A0685B05C01807F0FEF800258823D1
:1047400029008022A0685B05C01840196944520006
:1047500007F0EAF980230135FF355B019D42EED178
:10476000A6603E60044B9D44F0BDC046FCEFFFFFD9
:104770002C43FF1F9808FF1F04100000F0B5040031
:1047800087B0002825D0684607F0E6F81B4C0228C1
:1047900006D106226946200007F056FA002816D0F6
:1047A0006946002301250F262F00E25C0133100922
:1047B0001030874038002F00324097403A000243C3
:1047C0004A610439062BEFD16846FFF793FF07B023
:1047D000F0BD182269460A4806F0CEFF6A46A300DB
:1047E000D358013305D01822FF21684607F0DCF9C1
:1047F000EAE70134062CF1D1E9E7C0466509FF1F5D
:1048000000090011F0B5002504000E0085B0AA4291
:1048100000D186E04B1C087801934B788978377972
:1048200009021943F3783F061B040B431F43039708
:1048300020706570252800D196E033D8112813D850
:1048400007F092F869002501250125012501AA003C
:10485000B800B1002501250125012501250125010B
:104860002501250105011F01232800D1DEE0DB28F9
:1048700000D02EE1042A00D8ACE01025052A05D08E
:10488000551F2A003800711D07F036F90522310046
:10489000200007F031F92A003900601D07F02CF9DB
:1048A00005353EE0562859D010D8332800D19DE078
:1048B000552839D02628DAD19C4B2900132218001C
:1048C0001D0007F071F9FEF79BFB5CE0712800D139
:1048D00077E0722800D180E0602800D18BE0DC28EE
:1048E000C5D1022A00D875E07378BFB26370B3787F
:1048F000A370032A05D0033A390092B2F01CFEF7E8
:1049000083FC10223900E01CFEF744FDC51C002882
:1049100007DA60705CE00C222000854907F0ECF8B3
:104920000C25280005B0F0BD013A824D0C2A13D8A1
:10493000002A0AD02800019907F0DEF8FFF756FE9A
:104940000C2228007C49FEF75FFC29000C22601C29
:1049500007F0D2F80D25E4E70C22EBE7754D774B15
:104960002A0043CB43C2E9E7013A704D0C2A11D823
:10497000002A08D00199280007F0BEF80C22280070
:104980006F49FEF741FC29001322601C07F0B4F8C0
:104990001425C6E70C22EDE706226A49601C07F0E1
:1049A000ABF80625BDE712226749601C07F0A4F8A2
:1049B0001325B6E708226549601C07F09DF8092514
:1049C000AFE77178F02905D8614B188801F0BCFD7C
:1049D0000225A6E7FF236370FAE75E4B012A03D0A6
:1049E00072789A706270F3E79B78F4E72000FFF723
:1049F000E3FA050095E7013A564B574D062A10D8C1
:104A0000002A10D0012128005970019907F074F88C
:104A100001F056F829000622601C07F06DF8072502
:104A20007FE70622EEE700225A70F3E7042A04D952
:104A30004A4D2F6006F0B0FEA860FFF797FD0422F4
:104A4000039003A9601C07F057F8052569E7444D5A
:104A5000062ADFD906222800019907F0F5F8002878
:104A6000D8D006220199280007F046F806223D49D1
:104A70002800FEF7C9FB0123364A91780B43937057
:104A8000C8E7012AA6D07078FFF778FEA0E70128D2
:104A900000D0ECE6931E344F132B06D87378002B0E
:104AA0000BD100F015F900F04BF9304B39001D78AF
:104AB000601C6A1E07F020F833E7551E2A00019992
:104AC000380007F019F838002949AAB2FEF79CFB14
:104AD000E9E7DA281DD1042A00D87BE7082A15D98E
:104AE000B37972791B021343F27912041A43337AB1
:104AF0001B0613433B603B680522310020000393F3
:104B000006F0FAFF0422601D03A956E7FE23637036
:104B1000F1E7DE2800D05DE7511E012A01D1002512
:104B2000FFE6019800F0B2FFF9E7C046A061FF1F61
:104B3000ACBD0011D461FF1FFC0C0000A0BD001132
:104B4000F50C0000AC61FF1F8C61FF1F3043FF1F9D
:104B5000F041FF1FD061FF1F8D42FF1FE061FF1F6B
:104B60006509FF1FADAC0000D163FF1FCF63FF1FBE
:104B7000AEDE000070477047020010B5094B0A32E4
:104B8000094C92B2DA815A8298811882207802F018
:104B900041FB0422054B012120781A7006F064FEC7
:104BA00010BDC046BA42FF1F1A64FF1F1964FF1FE1
:104BB000013870B5042809D807F01EF80309280841
:104BC0001200234B0221187806F04EFE70BD204BD8
:104BD0000821187807F030F800221E4B1A72F5E70A
:104BE000802200241B4B1A4D52001A8108211A689A
:104BF0002878DC7206F050FE2100287806F0E4FFE9
:104C0000012000F07BFE00F05BFFDFE7104B082186
:104C1000187807F011F81048FFF76CF80F4B104A9E
:104C20009B79002093800F4A13808022094B520009
:104C3000D8721A8100F062FE00F042FF0A4B9B78A6
:104C4000002BC3D0094A136006F0A6FFBEE7C0469A
:104C5000F061FF1FC461FF1FF941FF1FD461FF1FF7
:104C6000BC43FF1FEA41FF1FD061FF1F34F000402B
:104C700010B501290BD1082809D1054B1B78002B51
:104C800005D02622034B04485A72FFF775FF10BD6A
:104C9000F263FF1FC461FF1FC40900000300F0B5E9
:104CA0000A4D8E18B14202D152008018F0BD0C7826
:104CB0002F6824093C5D0F271C700C7801313C40A3
:104CC0002F683C5D5C700233ECE7C046E441FF1F97
:104CD0000D22124B10B51A700C23114C1149237080
:104CE000093A033B1048637006F006FF2D230122AA
:104CF0000E490F48A371FFF7D1FF01220D49FFF7BD
:104D0000CDFF01220C49FFF7C9FF030000200B492A
:104D100002001870FEF778FA10BDC046EE63FF1F60
:104D2000CF63FF1F53BD0011D163FF1F6709FF1F32
:104D3000D663FF1F6609FF1F6509FF1FAEDE000077
:104D400070B5134C142220001249FEF723FB431EBA
:104D5000114D132B19D8AB78002B16D0431C2B7098
:104D600009236B7000230019037028780B4B013066
:104D70002900C0B2187006F067FD297822000139B9
:104D8000C9B2002005F0F4FD70BDFFF7A1FFECE70C
:104D9000D163FF1FAEDE0000CF63FF1FEE63FF1F76
:104DA00010B5114B1A781870002A0ED000280BD1BC
:104DB0000E4B1A78062A07D85423D340DB0703D5B5
:104DC0000B4B187802F026FA10BD0028FCD0074BD8
:104DD0001B78012B02D0033B022BF5D8044B012199
:104DE000187806F041FDEFE7F263FF1F1964FF1F1B
:104DF0001A64FF1F70B5514E514A52493070082055
:104E000005F042FC0121022005F048FB022005F0DC
:104E100029FC0121002005F041FB002005F022FCC7
:104E200000F0D2FEFEF7ECF806F05EFD03224649E4
:104E30004648FFF733FF2D24030004221C70444929
:104E40000130FFF72BFF30230470424D424C43707A
:104E500083702E3B062220004049EB87FEF79AFA2A
:104E6000062813D0200006F077FD022809D0032180
:104E7000200006F0D1FD8D23E3706E3B23711933C2
:104E80006371062220003549FEF7BEF9344B1B68DA
:104E9000FC335C64FFF754FF0020FFF781FF314CC7
:104EA000314A0121314B1278207802F075F9304AED
:104EB000304B12780021207802F06EF901222E4B3F
:104EC0001A702E4BDB78552B31D12D4B3B325A7259
:104ED0002C4B2D4AAB81EA812B826A8220213078CB
:104EE00006F052FE0120404205F08EFD01204042B6
:104EF00005F02AFEFFF710F9FEF7C4FE00F0B2FC41
:104F000001204042FEF79AFF012006F055FEF020F6
:104F100001F0FEFA0121307806F0A6FC307802F0AC
:104F2000D5FA1A4806F090FDFEF766FD70BD6422C2
:104F3000174B5B7953431A000A32CBE7F061FF1F2E
:104F4000754B0011714C00113043FF1F8C61FF1F26
:104F5000AC61FF1FBA42FF1F6509FF1FADAC000027
:104F60004464FF1F1A64FF1F1842FF1FF941FF1F0F
:104F7000EE63FF1FCF63FF1FC063FF1FD061FF1FE2
:104F8000C461FF1FC4090000CE090000F261FF1FC9
:104F9000D461FF1FF8B50A0020230D001A40194202
:104FA00063D05E4B1B78002B5CD0FFF7DFFA5C4BC5
:104FB0005C4C5D4E99686268737A8A1ADB039A4288
:104FC00002D36160FEF718FD327A217A531EDBB2FC
:104FD000994205D1FFF738F9002000F0A7FD15E050
:104FE0009142F9D300272772FFF758F9A37ABB4201
:104FF00002D0A772FEF788FD012000F097FD4B4F0D
:105000003800FEF777FE390006F09EFC637A002B2D
:1050100025D0013BDBB26372002B20D1444BDB78FF
:10502000552B01D106F0B8FDE37A002B12D00023F6
:10503000A27AE3729A4202D0A372FEF765FD3D4A5E
:105040003A4F1388380001331380FEF753FE3900BE
:1050500006F07AFC642370795843FFF78DFD237ABC
:105060000133237220206840F8BD0BB2002B0ADA0E
:10507000314B187806F008FD002801D006F01CFB23
:1050800080200002EFE70224214206D0254B0120B8
:105090001A72FFF785FE2000E5E70B071ED5FFF724
:1050A00065FA1F4B1F49204C98684A68637A821A38
:1050B000DB039A4202D34860FEF79EFCFFF7EEF84E
:1050C000FFF7C2F8012000F031FD00F0E5FB236896
:1050D000DB0701D5FEF7AAFF0820C4E7CB0609D5F8
:1050E000FEF712FD0D4B1B78002B01D1FEF7DEFD04
:1050F0001020B8E70124214207D0104800F06CF8D6
:1051000006F05AFC00F0F8FCC5E704240800204033
:105110002142A9D0FEF7AEFEBDE7C046F263FF1FF5
:10512000E061FF1FC461FF1FD461FF1FF941FF1F32
:10513000D061FF1FB861FF1FF061FF1FDC41FF1F3F
:10514000F0B51B4B1B4F1B883A8804001A4E1B4DB1
:1051500085B09A420DD832889A420AD3184B1A88E1
:105160002B889A4205D1174A174B12881B889A42FE
:105170001BD0052001F022FA3B8802AA1380338855
:10518000019053802B88114D93800F4B02A91B88EF
:10519000D3800F4B2A78188802F03EFF0D4B082170
:1051A0002878019A1C7006F0CFFA05B0F0BDC04611
:1051B000BE63FF1FEE41FF1FEC41FF1FEA41FF1FCF
:1051C000BC63FF1FBA63FF1FE841FF1F1A64FF1F84
:1051D000F041FF1FB863FF1F13B50C4B1C78002C68
:1051E00011D1002801D00A4B18600A4A0A4B1178E5
:1051F0000A4A10780A4A01920A4A0092002205F0EF
:10520000AFFA200016BD1124FBE7C0461964FF1F4A
:10521000B463FF1F1864FF1F0864FF1F1A64FF1F99
:10522000F463FF1FF863FF1F10B5064B12201B78B5
:10523000052B06D1044B13221988044B187801F072
:1052400099FB10BD1964FF1FF041FF1F1A64FF1F77
:1052500010B500240122114B52421870104B1C70E3
:10526000104B1A8002F032F904220F4B21001A7001
:105270000E480C3206F030FA102221000C4806F0DD
:105280002BFA07220B4B1C600B4B1C700B4B1C703A
:105290000B4B1A700B4B1C7010BDC0461A64FF1FDD
:1052A0001964FF1FF041FF1F1864FF1F0864FF1FF0
:1052B000F863FF1FF463FF1FCE63FF1FCD63FF1F63
:1052C000F241FF1FCC63FF1FF8B5174C060025788D
:1052D00006A814240078052D23D1B41F134FA5B2BE
:1052E0001824BD421DD88D1FADB2BD4219D8FA2574
:1052F0006D00AA4215D21D000D4F0A3DADB2BD4250
:105300000FD80C4C26800C4C21800C4900240A80BC
:105310000B4A1380FFF714FF0A4B0421187806F09C
:105320008BFC2000F8BDC0461964FF1F790C0000FB
:10533000750C0000EE41FF1FEC41FF1FEA41FF1F0B
:10534000E841FF1F1A64FF1FF0B50BB20D0089B0D2
:10535000002B00DB70E1A44E307806F095FB041EB4
:1053600050D00378A22B00D122E1D02B1AD0912B60
:1053700045D143780E2B42D19C4B82889A423ED134
:105380009B4A83681278052A39D1032018567F2852
:1053900035D0984B1B68002B31D05B68002B2ED08A
:1053A00098472CE08078072829D806F025FC0428A7
:1053B000183F3F74A8D86378002B0CD101218C4B87
:1053C00019708D4B1A78002A5BD08C4B307801F025
:1053D000E3FE002855D00722854B1A7051E0617812
:1053E0000029F8D1E378002B11D0854A854B12783B
:1053F000307801F0D1FE60706378002BEBD1200093
:1054000006F05AF980200002684009B0F0BD784BE0
:105410001B78022BF3D00121307806F02DFB0028F9
:10542000EAD10121307806F01FFAE5E76378002B16
:10543000D1D16F4F032807D13B78052B02D101331F
:105440003B701EE00223FBE76F4B1A886F4B029301
:10545000002A0BD01B78002B03D00121307806F0F6
:1054600073F93B78062B04D1013BE9E7029B1A70E4
:10547000F7E7042B41D10121029B3078197006F027
:10548000F3F95C4B1B68002BB9D01B68002BB6D01E
:10549000574A107884E76378554F002B27D10622AE
:1054A000211D5B4806F028FB62895A4B5A491A8035
:1054B000A2895A4B1A80E3890B800521397058491B
:1054C0000A80584A1380228A574B1A80574B1B7800
:1054D000012B09D11F2001F071F8FA2292004243FA
:1054E0000421307806F030F90022484B75E7312B63
:1054F00000D070E70022454B1A700323A0E7062274
:105500000021434806F0E8F80023454A04211380AF
:10551000444A30781380444A138006F08DFB0821FA
:10552000307806F089FBA379083B5A425341304A50
:1055300003331370304B1B78002B06D0334B30787D
:105540001A78002A06D001F065FE0122314B524242
:105550001A8096E70121197006F086F9F5E708210F
:10556000307806F069FB6378002B00D047E72C4BBE
:105570002D4F0293E388029A04211380294B30783F
:1055800003932389039A138063893B8006F074FA9E
:10559000002800D033E7264B1B68002B00D12EE7F4
:1055A000039902983A88098800881B68984726E77B
:1055B0004379132B00D022E70389012B0AD11D4B1D
:1055C0001B78022B06D10821307806F035FBFFF757
:1055D0002BFE14E7052000F0F1FF082102003078CF
:1055E00006F0B2F80BE7C0461A64FF1F051400006E
:1055F0001964FF1FB463FF1F1842FF1FF941FF1F0B
:10560000EE63FF1FCF63FF1FF063FF1FF263FF1FF7
:10561000C163FF1FF041FF1FC863FF1FCA63FF1F65
:10562000BE63FF1FBC63FF1FBA63FF1FC063FF1F82
:10563000B063FF1FB863FF1F8020C001014200D08C
:10564000E2E6CB0731D5324B1B78002B1DD0314E13
:1056500005AC3378052B1AD1023B23702E4B210069
:105660001B7823722D4B1B7863722D4B187801F039
:1056700037FD002809D007202A4B30701B68002B0B
:1056800003D01B68002B00D098470120BCE60E20F9
:10569000254B06221B7825492370254B1B78637008
:1056A00002ABC01806F028FAD8E702230800184019
:1056B000194209D0174B1B78052B03D11D4B1888B5
:1056C00006F072F802209FE60424214203D0FFF77F
:1056D00037FD200098E6082308001840194200D141
:1056E00093E6154B1C78012C03D0022C0DD008201A
:1056F0008AE6124B124A134913481B8812880988FC
:1057000000880094FFF7E0FDF1E7FFF78DFDEEE77D
:10571000F263FF1F1964FF1FF241FF1FCC63FF1FDD
:105720001A64FF1FB463FF1FCE63FF1FF341FF1F07
:10573000CD63FF1FF041FF1FB863FF1FE841FF1F4C
:10574000EA41FF1FEC41FF1FEE41FF1F10B502A809
:1057500004880B20002C10D1496808784978090288
:1057600001430C48814209D1022119800A4B598812
:105770001170DB7800205BB2537010BD074C0A201B
:10578000A142FAD102211980034B998811705B79EB
:10579000F0E7C0466E2A0000B861FF1F6F2A0000C4
:1057A000F7B5150008AA16884A680F4F1478527882
:1057B000120222430A24BA4214D10122DBB201921E
:1057C00000962A0005F0D2FE041E0BD1074B1B6881
:1057D000002B07D068782A780002104342425041DB
:1057E000013098472000FEBD022900002C64FF1FF5
:1057F00030B5012503790400BFB02B4225D01449F0
:10580000408805F01FFA28420CD0124B01A95B8D8D
:1058100000220B8002234B800F4B5B888B806088BB
:1058200002F0F0FA0D49608805F00CFAC0070CD5BB
:105830000B4B01A91B8800220B8002234B80064BD7
:105840009B888B80608802F0DDFA3FB030BDC04697
:105850002464FF1F1C42FF1FB861FF1F1C64FF1F51
:105860007642FF1F10B5074C0749200005F0A0F94C
:105870002000064905F09CF90721054A054805F076
:1058800059F910BDFFFF00002464FF1F1C64FF1FB7
:10589000CCBD00111C42FF1F10B5024803F034F9C3
:1058A00010BDC046F157001170B55F2508260749A5
:1058B0008400CA788B7840012A40B3433440A8431F
:1058C000234302438B70CA7070BDC0468D42FF1FD8
:1058D000010043B204205A0002409B000C300340F8
:1058E0001A43152310B5044CE0789843143B0B4041
:1058F00018430243E27010BD8D42FF1F10B5054BE7
:10590000082419790A00A243002801D022000A4382
:105910001A7110BD8D42FF1F10B5054B4024D97878
:105920000A00A243002801D022000A43DA7010BD09
:105930008D42FF1F0821F8B5324D334BAE7804007D
:105940000E40AE70984204DD67232B70473B6B70AE
:10595000F8BD2E4B984203DAE0232B703A3BF6E772
:1059600000232B706B7083B21A0029485F3292B209
:10597000284F82422CD9002C03DA5B421CB204234C
:105980002B70053420B20A2105F056FE04B2FA232A
:105990009B009C4232DB08232A7813432B7064213E
:1059A000200005F049FE0A2100B206F0D5F809B240
:1059B0002A787B5C13432B700A21200005F03CFE03
:1059C0000A2100B206F0C8F809B27B5C6A780AE0E6
:1059D0006970002CDBDA5B421CB204232B70F322CB
:1059E0006B78092CE8DC13436B700A21200006F069
:1059F000B3F809B27B5C1E43AE70A9E7632CCEDC22
:105A0000EDE7C0468D42FF1F1B4E00001DFCFFFF4F
:105A10002A080000F6BD00110823F7B5194FCD0084
:105A20003E7904001E403E71EDB2632806DD5F330F
:105A300033433B7120231D437D71F7BD03000933C0
:105A400005DA20235B4233433B71A623F3E70E4B79
:105A5000019300280BDA0423444224B23B710A214B
:105A6000200006F079F8019B09B25B5CE3E70928A6
:105A7000F5DD0A2105F0E0FD019B00B21B5C1E4331
:105A80003E71ECE78D42FF1FF6BD0011F8B50A4FDD
:105A900005003B780E00002B0CD0084C2000FEF7D0
:105AA0002FFC33002A0020003978FEF71DFD20006E
:105AB000FEF764FCF8BDC0463764FF1F9442FF1F29
:105AC00070B50A4E0A4D06223100280006F0BCF8D7
:105AD000002809D0074C31000622280006F00CF8F7
:105AE00007212000FFF7D2FF70BDC0468D42FF1F87
:105AF0003164FF1F3064FF1FE622402110B50A4BBE
:105B00001A70403A5A703E329A70DA780A40DA7067
:105B1000082219791140053A0A431A71D7225A719D
:105B2000FFF7CEFF10BDC0468D42FF1F10B5002805
:105B300038D0214C0223E05E204B1B685B0632D537
:105B400009233221584305F077FD4130FF3000B280
:105B5000FFF7F0FE0520FFF7A7FE0422A35E184A18
:105B60006320934205DC32331800642105F064FDA4
:105B700000B20121FFF750FF237A002413222000F6
:105B80009A426041C0B2FFF7C7FE2000FFF7A0FEB7
:105B90000C4B1878053843425841C0B2FFF7AEFEAF
:105BA000FFF78EFF10BD0A21053005F045FD00B25C
:105BB000FFF7C0FE0320CEE7B861FF1FD461FF1FCF
:105BC000DD2600001964FF1F70B500250A4C200077
:105BD000A571FEF795FB10233E212000074AFEF732
:105BE00083FCA84200D13E35054B20001D70FEF716
:105BF000C5FB0123A37170BD9442FF1FE6BD0011D8
:105C00003764FF1F0200F0B501270A480A4E5118F9
:105C10008B1A002B00DCF0BD08241578430868407F
:105C200038404000805B013C58406D08002CF5D1A5
:105C30000132EDE7FFFF000006BE0011F0B50025C0
:105C40000F269D4200DBF0BD4C5D07094440344007
:105C5000A400A05801357840F3E70000F0B589B002
:105C60006A460D000B000F27110010351C78013318
:105C7000260024093E40167054700232AB42F5D122
:105C80002023024AFFF7DAFF09B0F0BD0CBE001175
:105C9000F0B54E780B7889B036020C0017000190F1
:105CA0001E43012A61D9954B9E4200D877E001330B
:105CB0009E421CD1062A17D1CA788B7812021A4349
:105CC0000B791B0413434A7912061A438C4B5A6111
:105CD00000221A705A808B4A5A608B4A9A608B4A0B
:105CE000DA60002009B0F0BD88225205EEE7884B4B
:105CF0009E423CD182498B78002B00D0F6E00C2AE2
:105D000031D10F22A3789343E27812021343227910
:105D1000120413436279120613434B60E279A079AF
:105D200012020243207A00041043627A12060243F0
:105D3000CA60E27AA07A1202024376484A8183421C
:105D400008D804236E49142201980B7005F0D4FE84
:105D50001420C7E71201D21889235B059A42F0D8B4
:105D600001238B70BDE7022AFAD00523EAE76A4ACD
:105D700001239642E6D1FFF757FA052F0CD9E378B5
:105D8000A2781B021343227912041A4363791B067B
:105D90001343624A0393136005F0FEFEA1E7584DDA
:105DA0002B78002B9DD1AB78002B00D1A0E02B8964
:105DB00001339BB20093B34200D091E0132AD4D9AF
:105DC000CF7C8B7C3F02122120001F43FFF71AFF7C
:105DD000874200D08EE0002E3DD1E378A2781B02EE
:105DE00013432279E96812041A4363791B061343AB
:105DF00003930A228B4212D1FF23A370E370237115
:105E000063716B89002B09D1E37B227C1B02120496
:105E10001343A27B13431B0901336B8100226B895F
:105E2000002B8ED0002A67D1686837013818000B24
:105E30006B6900030390984205D9686105F07CFD09
:105E4000EB780133EB7068681022A11C381805F05C
:105E50006BFE2E8145E76F89009A7B1E9BB29342B1
:105E60003AD1E278A37812021A43237905A81B04D9
:105E7000134362796C6812061A43EB68009203922E
:105E8000211D0C22049305F037FE0120260004A9F1
:105E900040421036FFF7E2FE013F012F17D1009A72
:105EA0000B232861824200D04CE704221C492000C9
:105EB00005F03AFE042203A9686805F05DFCE96874
:105EC000039AFF23914200D13CE7F73B3AE73100C8
:105ED000FFF7C4FE1036DFE70923B742A4D831E745
:105EE000009BB34200D9FCE607232BE7022329E7F6
:105EF000032327E7062325E70A2323E7FFFE000005
:105F00009C42FF1F00000111FFFF0000504859365E
:105F100001FF0000FFFF001102FF000034F000400D
:105F2000A842FF1F10B5034C0B000122210000F016
:105F30006BFA10BDE56000110B8870B506000D000E
:105F40000224162B11D92B000322094900F05CFA18
:105F5000041E0AD1074B2A881B88191C934200D9BA
:105F6000111C300089B200F0EFFA200070BDC0466D
:105F7000116100114A64FF1F10B54A780400013A0C
:105F80000B000220012A07D80A78002A04D0052233
:105F90002000024900F038FA10BDC0463F610011F0
:105FA0000A7810B50B0004000220002A04D0072252
:105FB0002000024900F028FA10BDC046EB61001134
:105FC0000A7810B50B0004000220002A04D0092230
:105FD0002000024900F018FA10BDC04651620011BD
:105FE00010B5034C0B000B22210000F00DFA10BD80
:105FF0008162001110B5034C0B000D22210000F04E
:1060000003FA10BDF362001110B5034C0B000F2210
:10601000210000F0F9F910BD4D6300110A7810B5A8
:106020000B0004000220002A04D0112220000249A3
:1060300000F0EAF910BDC0465D630011002310B501
:106040001322190000F0E0F910BD000010B5034C58
:106050000B001722210000F0D7F910BDAF6300112B
:10606000002310B51922190000F0CEF910BD000070
:1060700010B5034C0B001B22210000F0C5F910BD28
:10608000E9630011F7B584890D0006000121002C99
:1060900022D000238268D3561778002B1EDA0C2CEE
:1060A0001AD90C3CA4B2131940880093230002F0C3
:1060B00086FE431E984101307B06DB0F6B703F2349
:1060C000013C1F40A4B22870AF70AC80002C07D0F8
:1060D000B3680133AB6000210800FEBD0020EBE790
:1060E000AC60F8E70B7803704B8843704B881B0A51
:1060F00083700B79C370042070470420022B06D1F3
:106100000020537811781B02009A0B4313807047CC
:106110000B8803700B881B0A437002207047042011
:10612000009983420AD1537810781B0203430B80F5
:10613000D37890781B02034300204B807047F8B55A
:106140000D004B7801240021461C03702B788B42F4
:1061500001D82000F8BD6B78B01C4F1C012B10D16A
:10616000890069184B88022233704B88B9001B0ADA
:106170007370691805F080FA04360434A4B2F9B2D9
:10618000E4E7122359436B185A88043132705B8854
:1061900010221B0A7370691805F06EFA1236123459
:1061A000ECE770B5049D14001E00052B01D80420F7
:1061B00070BD637812781B0213432B80E378A278BA
:1061C0001B02134302226B802A71211D681D063EAB
:1061D00005F052FAB2B22A81E92AE8D82800A11DB6
:1061E0000A3005F049FA0020E2E7002310B50A78EA
:1061F0009A4201D8900010BD9A008A185488013341
:1062000004705488DBB2240A4470948884709288A5
:10621000120AC2700430EAE710B51100029C062B86
:1062200004D004201022142B01D010BD02222271B0
:106230004B7808781B0203432380CB7888781B02B5
:10624000034363800431601D05F016FA0020ECE77B
:1062500010B50C788B7804315C43E4B203702200F3
:10626000013005F009FA601C10BD0420022B06D194
:106270000020537811781B02009A0B43138070475B
:1062800010B50C000A88023105F0F6F9208810BD1F
:1062900070B504000D0004981100012B01D80420F2
:1062A00070BD167852781202324302800200F13239
:1062B00055701470E125002C00D10C35023B9AB2C8
:1062C0004280AA42EBD80231043005F0D5F9002013
:1062D000E6E70420009983420AD1537810781B0224
:1062E00003430B80D37890781B02034300204B803C
:1062F000704710B50C000A88023105F0BDF92088FE
:1063000010BD000070B501211E000420049C0E4049
:106310000B4218D1CB40DDB28D4214D90A49DBB211
:10632000098899420FD32300EE331D7033005800C3
:1063300011184978165C0902314301332152D9B250
:106340008D42F4D8002070BDB442FF1F10B50C0080
:106350000A88023105F090F9208810BD10B50C783C
:106360008B7804315C43E4B203702200013005F005
:1063700083F9601C10BD10B511000298032B01D8E1
:10638000042010BD14785278043B1202224302808C
:10639000CA788C781202224342809AB28280EB2A19
:1063A000EED80431063005F067F90020E9E710B5B2
:1063B0000C000B8803700B881B0A43704B8883709A
:1063C0004B881B0AC3708A880430063105F054F9E3
:1063D000A088043080B210BD0420012B03D100201E
:1063E0001378009A1370704710B50C000B88037077
:1063F0000B881B0A43704A880230043105F03CF9CF
:106400006088023080B210BDF0B589B003931E4B96
:10641000029242000700D05A019102F020F81325A1
:10642000061E2DD0029B01240370019B002B04D07B
:10643000001903999847001984B26B461B7A5BB226
:10644000002B0FDA1021380002F01CFB1925002860
:1064500013D130003219E1B202F066FC051E0CD1F6
:106460000C34A4B2042304AA380005A9938006962C
:10647000948101F0AFFD051E02D0300005F0CCF98B
:10648000280009B0F0BDC0464864FF1F70B5050084
:106490000C0000280CD00020814209D010222000DE
:1064A000044905F0E9F801202B7823736B786373B6
:1064B00070BDC0464CBE0011F0B506000D001700BF
:1064C0001C0085B002291BD00020102907D1022B07
:1064D00007D0102B03D115E00020102C08D005B0F8
:1064E000F0BD69463800FFF7D1FF2A0069460BE08E
:1064F00069463000FFF7CAFF22006946380004E011
:10650000022BE9D12A003900300005F035FBE6E71F
:10651000031CF02800D9F023032008499AB2013A5D
:106520000B80D317034006499B189B100B80D30F99
:1065300004499B185B100B807047C046B842FF1F90
:10654000B642FF1FB442FF1F034B1B888B4202D38E
:10655000024B4000C1527047B842FF1F4864FF1F02
:10656000014B4000185A70474864FF1F1722014B27
:106570001A8070474864FF1F70B505000E2005F0B3
:106580004BFB041E13D0D02303700023062283701C
:1065900007494570033005F06FF8064B2100DA8A91
:1065A00062811B7E2373044B187805F06DFB70BD70
:1065B0006464FF1F5464FF1F0843FF1F262803D88D
:1065C000024B4000C05A70470148FCE7BA42FF1F27
:1065D000FFFF000070B506000C00094D1C220021D1
:1065E000280005F079F8074B1E70074B1C7005F06A
:1065F00073FA0123002801D0002312202B7070BDF4
:106600005464FF1F0843FF1F7564FF1F70B505002A
:106610000D4C0800E260A16010220021656005F0C9
:106620009BF8012803D11021A06802F058FD102228
:106630000021280005F090F8012803D1102160689E
:1066400002F04DFD70BDC0465464FF1F70B5041EBE
:1066500005D1002903D006220D4805F00DF80D4B99
:106660001D78012D11D1002C05D102221A7004F0E1
:10667000FBFF280070BD00221A70074B1B78FF2B10
:10668000F7D02000FFF778FFF3E70025F1E7C046D9
:106690006464FF1F5464FF1F0843FF1F030010B50D
:1066A000002801D1002010BD00780B4A002803D13A
:1066B0005988D1821B7913761378022BF2D10023EB
:1066C000984200D103331370044B1B78FF2B01D089
:1066D000FFF752FF0120E6E75464FF1F0843FF1F46
:1066E000002911D000280CD04B79012803D1402279
:1066F0005242134303E03F221340032802D00120FB
:106700004B7170474022F4E70800FAE770B5094D75
:106710000100287800280BD0074C0622200004F046
:10672000ABFF21002878FFF7DBFF200005F0FCF825
:1067300070BDC0467464FF1F4E64FF1F00290AD05D
:10674000012808D13F224B799343C02B03D0403B13
:106750005A425341981C704770B5174D06002B786C
:10676000FF2B15D00A2005F057FA041E10D0D023B5
:106770000370C83B8370114B11491B784670C3707E
:106780000622043004F078FF2100287805F07CFA16
:106790000C4B1B78012B0DD10B4B1B68002B03D02E
:1067A0009B68002B00D09847084B04211878084AB2
:1067B00005F072F870BDC0460843FF1F7464FF1FE8
:1067C0004E64FF1F7064FF1F9C64FF1FA064FF1FC7
:1067D00060EA0000014B98687047C0465464FF1F90
:1067E000014BDB68186870475464FF1F074B10B5F6
:1067F000DA68136801331360054B1878FF2803D05B
:106800008021C90105F030F810BDC0465464FF1F57
:106810000843FF1FF7B50E0002F0C8F8051E1CD094
:106820000E4B06621F78002F00D10778AB7910203D
:10683000019305F0F1F9041E0FD0D0230380C73B6C
:106840008370019BE91DC3700622043004F014FF1D
:1068500021003800E66005F017FAF7BD0643FF1F78
:10686000014B18787047C0467464FF1F054B002821
:1068700005D1054B1A78054B002A00D1014B1800B1
:106880007047C0466464FF1F7464FF1F4E64FF1F9F
:10689000014B58687047C0465464FF1F024B18688C
:1068A000431E9841C0B270477864FF1F421E030028
:1068B0000120152A03D9FF3B5A425341D8B27047F1
:1068C000F0B51C0000230E0085B0039002920B70FF
:1068D000029A934201D3002019E0E55C5A1CD2B21F
:1068E000002DF8D0029851198142F4DC0233DFB256
:1068F000A35C18000193FFF7D9FF002807D0013DE2
:10690000019A0399EBB233708A4202D1E01905B0C3
:10691000F0BDDB19DBB2DBE710B50C0002F09EF82E
:1069200003001220002B03D02100588804F0A4FF9C
:1069300010BD000070B50E4D84006359002B15D0BA
:10694000186A002801D004F0AFFE2B59586A0028BD
:1069500001D004F0A9FE2B59986A002801D004F058
:10696000A3FE285904F0A0FE00232B5170BDC046A1
:106970008464FF1F1C4B70B504000E001500994283
:106980000AD11A4B1B68002B01D1122070BD1B6865
:10699000002BFAD09847F9E7154B994215D1134BC4
:1069A0001B68002B0AD01B68002B07D098470028D3
:1069B00004D1104B1C70104B1D70E7E7290020001C
:1069C000FFF7AAFF0028E1D1F3E7080001F0EEFF8E
:1069D0000028DAD003780320A342D7D12900300061
:1069E00004F04AFFD2E7C046FEFF00008064FF1FAC
:1069F000FFFF00007D64FF1F7C64FF1FF7B50400EC
:106A0000808801F0D3FF0025A84203D00578A08834
:106A100002F008F81C4E3378002B1FD0AB421DD17A
:106A20001A4B28001978FFF777FF002818D00023A9
:106A30003370A3790820A778A688019305F0ECF8B5
:106A4000011E0DD0D0230370CA3B8370019B477099
:106A500086808371280005F017F901E0002DE8D148
:106A6000A0880B4B8200D358002B01D0FFF762FFA8
:106A70001721A088FFF768FDA08801F027FDA088F6
:106A800001F0FEFDF7BDC0467D64FF1F7C64FF1F63
:106A90008464FF1FF0B587B01D000CAB1B88070096
:106AA00001930DAB1B88142002930EAB1B881600BC
:106AB00003930FAB1B880091049310AB1B880593C5
:106AC00005F0AAF8041E1AD0D0230370CB3B477000
:106AD0008370C670062229000430002D11D004F006
:106AE000CBFD019B21006381029B0098A381039B46
:106AF000E381049B2382059BA37405F0C5F807B0CE
:106B0000F0BD04F0E9FDECE7F7B5009308AB1B8896
:106B100007000C200D001600019305F07DF8041EFF
:106B200013D0280001F042FF00280FD00078D023B6
:106B30002370C93BA370009B21002381019B6770D8
:106B4000A580E680638105F09FF8F7BD014B1878BA
:106B5000EDE7C0460843FF1F13B5040064890389AD
:106B6000C2888188C0780094FFF7CEFF13BD000073
:106B700010B5044C2068002803D004F095FD0023D4
:106B8000236010BD8864FF1FA122F0B581889200A8
:106B90004A43384B384F1B6804009B189D229200D3
:106BA0009B18827989B01A603B68002B5FD01D78F2
:106BB000324B1B68002B04D05B68002B01D00020F7
:106BC0009847260008363100E079FFF7B7FD237DAE
:106BD000E0710200E0780493638A29000393238A1A
:106BE0000293E3890193A38800933300FFF752FFD8
:106BF000E378002B0BD1E289A379A1880292019658
:106C0000E27928000092012201F0DAFEE0703B6890
:106C1000002B20D0FFF7ACFF194D287800281AD0A0
:106C2000184B1978FFF778FE002814D02B78E678F7
:106C300008200793A78804F0EFFF011E09D0D02396
:106C40000370CA3B4670837087808671079805F091
:106C50001BF800232B701721A088FFF775FCA08874
:106C600001F034FCA08801F00BFD09B0F0BD064B2B
:106C70009DE7C0463409FF1F8864FF1F9C64FF1F07
:106C80007D64FF1F7C64FF1F0843FF1FF8B50700EA
:106C900008000E0001F08AFE041E18D02620FFF71F
:106CA0008DFC051E00D12578062004F0B5FF041EDA
:106CB0000DD00021062204F00FFDD0232370C23B2B
:106CC00021006770A370A680E8B204F0DDFFF8BD74
:106CD000F0B585B001930AAB1B78070002930BABAC
:106CE0001B7808000D000092039301F05FFE061E62
:106CF00022D0102004F090FF041E1DD0102200218D
:106D000004F0EAFC2620FFF759FC002800D1307877
:106D1000D0232370C13BA370009B21002372019BF1
:106D200067706372029BA580A372039BC0B2E3727B
:106D30000C9BE36004F0A8FF05B0F0BDF7B50D00B3
:106D4000019001F033FE071E20D00E2004F064FFF6
:106D5000041E1BD02620FFF731FC061E00D13E7812
:106D6000D0232380C53B0622A370F91DE01C04F04C
:106D700083FC019B2A0063810123DD401A401D40F2
:106D8000210022736573F0B204F07EFFF7BD0000AE
:106D9000F0B585B0029010000D0017000A9E039315
:106DA00001F004FE041E31D0029B002B2ED1039B68
:106DB00002795B0724D5122313430422002E08D145
:106DC0000B99002905D10C99002902D10D990029B0
:106DD0001AD01A430D9B2271002B00D0C9E0002E5F
:106DE00000D1CFE0002D00D0CCE0606A002801D0B7
:106DF00004F05AFC1C21300004F0E6FC606205E05F
:106E000002239A430E33D7E793432371654BBA00AD
:106E1000D458002C00D1AAE0002E10D0236A002BF9
:106E200003D11C2004F080FC20625E4BBA00D358D2
:106E3000186A002803D01C22310004F01DFC0C9BB2
:106E4000002B12D0574CBB001D596B6A002B03D18D
:106E5000162004F069FC6862BB00E358586A0028F9
:106E600003D016220C9904F007FC0D9B002B11D0C7
:106E70004C4DBC006659B36A002B03D1142004F0BA
:106E800053FCB0622B59986A002803D014220D9944
:106E900004F0F2FB380001F089FD051E67D0414B7C
:106EA000BA00D358002B62D01A6A3420002A00D1CD
:106EB0001C389A6A002A01D0143080B20B9A002A3A
:106EC00001D01C3080B25B6A002B01D0163080B23A
:106ED00004F0A2FE041E4AD01822002104F0FCFB9C
:106EE0002620FFF76BFB0190002801D12B7801933E
:106EF000D0232370029B200063700A23294EA370C5
:106F0000039BBD00A371AB59A780196A18300029F3
:106F100005D01C22A06004F0AFFB20003430735970
:106F2000996A002907D0030014221433E060029309
:106F300004F0A2FB02980B9B002B08D003001C223C
:106F40001C330B992061029304F096FB029873594D
:106F5000596A002903D01622606104F08DFB6B464C
:106F60002100187904F090FE3800FFF7E3FC05B02B
:106F7000F0BD10220D9B0D991B69A018236204F02F
:106F80007BFB2CE70B9B002B00D13FE7012D00D0B2
:106F90003CE7606A002801D004F086FB1C210B98B6
:106FA0002AE7C0468464FF1F10B5044C20680028FF
:106FB00003D004F079FB0023236010BD7864FF1F29
:106FC0000B4B07B51A68002A01D100200EBD694697
:106FD000531C012012780731FFF772FC0028F4D00F
:106FE00002780123100018401A42EED0EEE7C046A6
:106FF0009464FF1FF0B51F4F01203B6887B0002B42
:1070000025D09B78059300F0B3FB002821D00A20FF
:10701000FFF7D4FA04000B20FFF7D0FA164B050057
:107020001E78731E9E413B68F6B2191DD878FFF793
:1070300057FB3B682900DA7A043303929A7901936B
:107040000292009033002000059A04F05DFB07B027
:10705000F0BDFFF7B5FF002805D00620FFF7AEFA18
:1070600004000720D8E70820FFF7A8FA0400092049
:10707000D2E7C0467864FF1F7464FF1F70B50A4EE4
:10708000040033780D00FF2B0DD0042004F0C4FD64
:10709000011E08D0D0230370CE3B45708370C470AE
:1070A000307804F0F1FD70BD1843FF1F70B5040087
:1070B00006200D0004F0B0FD011E0AD0D02303709D
:1070C000CD3B8370054B44701B688580187804F0B5
:1070D000DBFD002C01D0FFF767FF70BD7864FF1F58
:1070E000F8B5264F06003B680D001124002B05D192
:1070F0000522234B1B78134202D112242000F8BD35
:10710000204A10241268002AF8D01278002AF5D0FC
:10711000DB0719D52B789A1E012A1AD80C2004F007
:1071200003FB132438600028E8D000230A224370B0
:1071300029000670023004F09FFAFFF75BFF041E7F
:107140000AD0FFF731FFD9E700F012FB0028E1D1A8
:10715000E4E7002BE2D0D0E70B4B1B78032BCDD11B
:107160001D20FFF72BFA094B18800028C6D0084BCA
:1071700004211878074A04F08FFBBFE77864FF1FEB
:107180007564FF1F9464FF1F7464FF1F7264FF1F08
:10719000A064FF1F60EA0000F7B50193194B1400CB
:1071A0001A78052306000F0012201A4221D0012967
:1071B00020D1154B1D68002D1BD002201F2C18D884
:1071C000002C02D0019B002B13D0104B1F221E70ED
:1071D0006E1C0021300004F07FFA0199220030007B
:1071E00004F04AFA310020002C70002F06D004F081
:1071F00083FAFEBD064B12201D68DCE704F024FB79
:10720000F7E7C0467564FF1F9464FF1F1843FF1F14
:107210009064FF1FF8B50F4E12243368002B17D06F
:107220001B780F3C834213D100250B4F0221387885
:1072300004F002FD094B042138781D8004F0FCFCA9
:10724000074B28001D8033685C7004F0DDFC0400EF
:107250002000F8BD7864FF1FA064FF1F8C64FF1F2F
:107260007264FF1F70B5012823D11B4C2388002BAB
:1072700003D01A4A1578002D07D0194B1B68002B34
:1072800002D01878FFF7C6FF70BD3B2B02D93C3BFC
:107290002380F9E7134E0221307804F0CDFCFA2266
:1072A0002388920002215A43307804F04DFA258059
:1072B000EAE70B4B1B68002BE6D00B4B1B785B07F8
:1072C000E2D5084B0221187804F0B6FC0022024BEC
:1072D0001A80FFF769FED7E78C64FF1F7064FF1FF9
:1072E0007864FF1FA064FF1F7564FF1FF8B51E4D73
:1072F0002868002803D004F0D7F900232B601B4E28
:107300003068002803D004F0CFF900233360184F11
:1073100005243B7818002040234221D0154800F076
:107320002BFA3B78234213D0202004F0FDF928608B
:10733000002813D02022002104F0CEF9202004F0F0
:10734000F3F9041E306005D02022002104F0C4F9B6
:10735000002004E0286804F0A7F92C601320F8BD91
:1073600000F00AFAF4E7C0469464FF1F9064FF1F20
:107370007564FF1F0C43FF1F10B50A4C23681A1ECB
:107380000ED0002808D10130587004F03DFC0028D0
:1073900005D02368002B02D00021FFF787FE0122D1
:1073A000100010BD7864FF1FF7B5274E0500336845
:1073B0000191181E21D05C78244F012C30D1FFF7A9
:1073C000FFFD002825D02000FFF7F8F80400412831
:1073D00014D91F4B022118781E4A04F05DFA1E4B87
:1073E0003C3C1C80022233685A703B78002B14D13D
:1073F00028000199FFF75AFE0120FEBDFA229200F3
:107400004243002AEED0124B0221187804F09CF976
:10741000E8E7FFF7D3F80200F3E700233B70EBE760
:107420003B78002BE8D1032004F0F6FB011E08D0C6
:10743000D0230370CC3B457083703368187804F018
:1074400023FCFFF7B1FDD7E77864FF1F7064FF1FCF
:10745000A064FF1F60EA00008C64FF1F10B517498D
:10746000838802008B4220D011D815498B4217D057
:10747000144900205B1899B2012907D89268117845
:107480005A425341D8B2FFF7F9FD012010BD0E4A10
:1074900000209B1807229BB29A424041C0B2F5E7F8
:1074A00083681878FFF768FFF0E7836899785A785F
:1074B000090218781143FFF777FFE7E70A20000079
:1074C00006200000F8DFFFFFAFDFFFFF014B187061
:1074D0007047C0461943FF1F10B5064C207001F0DD
:1074E00041FA207804F080FB0521207800F062FD4D
:1074F00010BDC046A064FF1F0BB273B50D00002B7A
:1075000000DBC4E0884B187804F0BEFA041E0ED0ED
:107510000378912B0FD0A22B00D1A1E0834B1878D8
:10752000FF2852D0210004F0AFFB00284DD180206D
:107530000002684076BD43780F2B76D013D8052B18
:1075400070D00E2BEAD18088794B98422BD8794B9A
:1075500098421BD8784B9842E0D1A3681878591C00
:10756000FFF774F838E03E2BD8D18378032B74D022
:107570006CD8012B6ED0022BD0D1704B1B68002B26
:1075800023D05B68002B20D098471EE06C4BC018BE
:107590000C28C3D804F018FA1DC2C2150BC20B0B7D
:1075A0000B3223C23C00674BC0180728B6D8664B85
:1075B0001B68002B09D01B68002B06D020009847C1
:1075C0000AE0A3681878FFF7C7F8200004F074F801
:1075D000ADE7A068FFF762F800289FD0F5E7A36841
:1075E0001B78002BF1D0554B1B68002BEDD01B688E
:1075F000002BEAD0210055489847EDE74F4B1B6818
:10760000002BE2D01B68002BDFD021005048F3E7AD
:10761000504B1B68002BD8D05B68002BD5D02100C5
:107620004348E9E7FFF7EAF9CFE780884A4B9842F9
:1076300003D04A4B984200D070E7464B1B68002BA2
:10764000C3D05B68002BC0D02100D5E7153B012BD0
:10765000BBD963E7FFF798FAB7E7FFF77DFAB4E71E
:107660003F4B1B78042B07D100236A461380017916
:10767000408800F0C5FCA8E7364B1B68002BA4D05F
:107680005B68002BA1D00100364898479DE7012494
:1076900021420AD0294B1B68002B04D05B68002BC9
:1076A00001D000209847012043E78B070AD5264BDD
:1076B0001B68002B04D05B68002B01D0200098478A
:1076C000022036E70421280008400D4200D131E7AE
:1076D000254E3388002B21D0013B9BB23380002BF9
:1076E0001AD1FFF7DBF800280AD0204B1C70164B8C
:1076F0001B68002B04D05B68002B01D0200098474A
:10770000FFF7C6F8694601F001FD6846FEF7FEFF87
:107710001D20FEF753FF308004200AE7024B187843
:1077200004F08AFAF8E7C046A064FF1F1943FF1F60
:107730000E20000001200000091000009864FF1FC7
:10774000FEDFFFFFAFDFFFFF9C64FF1F0C20000088
:107750000B2000008064FF1F0D200000132000009C
:107760007564FF1FFFFF00007264FF1F7064FF1F3E
:1077700010B501F09BF910BD014B18607047C04671
:107780009C64FF1F0B880020162B01D817230420B0
:10779000014A13807047C0464A64FF1F00207047AB
:1077A000074A03001188814207D09188002099423E
:1077B00002D101308000101870470020FAE7C0465F
:1077C000A864FF1FF0B58F7806000D00C5B01E2F0E
:1077D00015D1FFF7E5FF051E03D10024200045B0B9
:1077E000F0BD00223B003100C078009200F0B2FBF7
:1077F0000400A81C00F0D2FBFF23EB70EEE7264B41
:10780000062403931B78FF2BE8D0182FE6D87B08BB
:10781000224A013BDB0002929A589446002ADDD0AE
:10782000029AD3185B68002BD8D00878002802D1C0
:107830004B78012B02D10624122FCFD107AFAB8892
:10784000697800976446AA68A047041EC6D1AB7841
:10785000029A5B08013BDB00D318390030005B68FB
:107860009847041E0BD1AB78042BB6D0039A310095
:1078700010782200009700F06DFB0400AEE76A78F4
:10788000002AABD1AA7805A93B88087130000A709C
:107890004B80FEF747FBA0E71C43FF1F5CBE0011B7
:1078A0001D4B37B5050098420BD000290AD1FFF7D0
:1078B00077FF002805D11948FFF772FF002800D094
:1078C000058037BD01291AD1FFF76AFF041EF8D0E1
:1078D00001235B420380A378FF2BF2D0FE2B07D05D
:1078E0000023E0781422009329001E3300F032FBBD
:1078F000A01C00F053FB01235B426380E1E70229F7
:10790000DFD1013901F0BEF80028DAD12800FFF7F5
:1079100047FF041EDFD1D4E7FEFF0000FFFF000099
:10792000022210B5074B52421A80074801325A8092
:107930009A80DA8000F07EFA044801F025F80020F1
:1079400010BDC046A864FF1FC5770011A1780011C3
:107950000388F7B50400002B02D102252800FEBDE4
:1079600042680221137825485268FEF7A5FD0028D9
:107970002ED0234F01253A88002AEFD0802321887A
:107980005B0201259B1A9942E8DC0C2003F0CCFE37
:10799000061E31D03B8822889C46002318000195A2
:1079A00061469DB2491989B2AA421BD8002801D06C
:1079B00062443A8000233000082208C0210003F00E
:1079C0005BFE104A1368002B13D100251660C5E733
:1079D0006268022113780C485268FEF76DFD00289A
:1079E000C7D1BAE760681D01401941810133019890
:1079F000D6E71A001B68E6E71325AFE7CABE0011F9
:107A00001A43FF1FA464FF1FC8BE0011014B18706A
:107A10007047C0461C43FF1F14230A0010B51A40CC
:107A2000194204D00122102101F048F810BD4B0684
:107A3000F9D4012088434000F8E710B514008B0604
:107A400004D50122102101F039F810BD08230A00E5
:107A50001A40194202D14BB2002B0FDA102101F06B
:107A60002DF8002808D02300F2331B78002BECD02F
:107A7000F1342378012BE8D10020E6E703208907C1
:107A8000FAD4E2E7F0B51F00184B85B01C680190EE
:107A900002910392002C27D1200005B0F0BDA5680B
:107AA0003301ED186B89019A934211D3029A9342E4
:107AB0000ED8002F04D10A9B002B10D12C00EBE72D
:107AC0003B002978039A6868FEF7F6FC0028F2D19B
:107AD0000136B6B2A388B342E1D82468DAE7A368D6
:107AE0000A9A5B891380E9E70026F3E7A464FF1F85
:107AF00037B50C000A8849880123914217D3002A20
:107B000015D0651D23792A0002210A48FEF7D4FC0E
:107B1000102300280BD023796188208800242A00B4
:107B20000094FFF7AFFF0A23A04200D02300180003
:107B30003EBDC046CABE001113B50A000888498878
:107B4000012388420BD8002809D00024137905327C
:107B50000094FFF797FF0A23A04200D023001800EB
:107B600016BD13B50A0008884988012388420BD83E
:107B7000002809D00024137905320094FFF782FF12
:107B80000A23A04200D02300180016BDF0B58BB028
:107B900003904A8808880E000123824255D30028AA
:107BA00053D00023012704AC2370002271881300F6
:107BB0000092FFF767FF051E3ED02078002835D1E0
:107BC0002B78022B18D167706A8983000130E31883
:107BD00080005A8069680222201803F04DFD237846
:107BE0000133DBB22370042B19D93B0068890130C3
:107BF00080B2002BD9D01FE00223637012235843B8
:107C00006A89231804305A8069681022201803F00A
:107C100033FD23780133DBB22370002BE5D10C4A0E
:107C20006B899B185A425341DBB2DFE76378012B23
:107C3000E4D12B78022BC7D022780A23002A04D063
:107C400021000398FEF798F9002318000BB0F0BD4F
:107C50000100FFFF0F4BF0B504001868002816D094
:107C600083685D89A54207D88288AE18B44203DADA
:107C700012019A18934201D10068EFE71E005F8954
:107C80001036A74204D1002900D00D801800F0BDA5
:107C90003300EFE7A464FF1F70B505000C000888EF
:107CA0000021FFF7D7FF03000120002B04D02200A2
:107CB0002800197AFFF7C1FE70BDF7B50C0000254A
:107CC00001902300EE331B78AB4201D800200AE07C
:107CD0006B00E65A00213000E718FFF7BBFF0028D1
:107CE00002D126800130FEBD017A0198FFF794FE93
:107CF000002802D03B882380F5E70135EDB2E0E7AC
:107D000010B5040008880021FFF7A4FF030001203C
:107D1000002B03D02000197AFFF77EFE10BD000073
:107D2000054B1B68002B01D1180004E09A685289AA
:107D30008242F6D198887047A464FF1FF0B50E27E1
:107D4000002687B0039302ABFF183E8005001F4B4F
:107D500040891400984207D02B78013000976A6858
:107D600080B2FFF78FFE060002212B7818486A6860
:107D7000FEF7A2FB00280FD06C892000FFF7D0FF90
:107D8000002802D0013C0419A4B2039B002B00D0B0
:107D90001C80300007B0F0BD02212B780D486A68C6
:107DA000FEF78AFB0028E7D102212B780A486A688F
:107DB000FEF782FB002807D0002EDED03B88A342CE
:107DC000DBD17489013CDFE76C89DEE7FFFF00004F
:107DD000CABE0011C8BE0011C6BE001110B50C000D
:107DE000FFF7DEFC03000220002B0AD0002C00D09D
:107DF00023609B781720FE2B03D00138FF2B00D186
:107E0000002010BD73B50D0001A904001600FFF796
:107E1000E5FF172805D0002E04D129002000FEF729
:107E200027F976BD01221021200000F047FE00282E
:107E3000F3D0F6E7014B18607047C046B464FF1FEB
:107E400037B56B469D1D010004000222280003F097
:107E500053FE2B88B02B0ED12379122B09D123008E
:107E6000FA331B78012B06D10121608800F0E0F87D
:107E700001E01B2BF8D037BD10B5054B042118705D
:107E800000F098F8FFF74CFDFEF770FB10BDC04600
:107E9000B864FF1F0020F0B50BB20F0087B083421B
:107EA00034DA274B187803F0EFFD051E2BD003784A
:107EB000A02B25D103AE3100FEF7E4F8041E0BD150
:107EC000B378DB0724D51F4B06341B68002B03D087
:107ED0003100688898470400A868002801D003F0A2
:107EE0009BFC002C08D1184A039B1340174A93426D
:107EF00006D0B3781B2B03D00121688800F098F8D6
:107F0000280003F0D9FB80200002784007B0F0BDC4
:107F10000F4B1B68002B10D0310068889847041E57
:107F2000DAD07378002BD7D1B27801A90A704B80D0
:107F30000C716888FDF7F6FFCEE70624F1E7C0462E
:107F4000B864FF1FB064FF1F00FFFF0000011200B4
:107F5000B464FF1FF7B50190FC200D0017001E0050
:107F600003F05AFE04001320002C12D0B02320008E
:107F70002370089BF4226770658026710830002BFF
:107F800008D0190003F078FB2100019803F07CFE73
:107F90000020FEBD089903F09FFBF5E710B5041E15
:107FA00006D00078FD2803D803F046FCFF23237099
:107FB00010BD00000A1F93B210B504000220032B6D
:107FC00005D882400020024BD1529B189C7010BDF6
:107FD000D864FF1F0B8870B5043B04000D0002201D
:107FE000032B0BD80121200000F04CFD03001420CE
:107FF000002B03D02900200000F0DEFB70BD000044
:1080000007B51300034A00920A00012100F02CFC7E
:108010000EBDC0463D82001107B5019203220092B9
:10802000024B0A00122100F049FC0EBDBB82001178
:1080300007B56B4601AA11800449D8800878063339
:10804000012802D1190003F09FFB07BDB964FF1F8F
:108050000C4B10B518700023FF210B4A13801381BD
:1080600093819380094A5380137051729381937264
:10807000D174D3821375517703F08EFC00F0FCF9B4
:1080800010BDC046E864FF1FD864FF1FBA64FF1F1D
:10809000F0B58DB06B46002003910C229B5E8342AD
:1080A00000DBB0E05D4B187803F0EEFC051E00D15C
:1080B000A4E00378902B00D09DE006AF0100468835
:1080C000380000F013FA79680400002900D19CE020
:1080D0003B88052B6ED13B89032B1CD905AC2000B6
:1080E00000F0A2F86288172A61D83989131D9942D5
:1080F00031D17968237804310291D90738D5607875
:1081000000F08EF9071E06D0002303712378012B9F
:1081100008D0132B23D0A868002800D178E003F002
:108120007BFB75E06288029909A800F0A6F802902E
:10813000380000F08BF909AA2378387A01920022DE
:1081400031000092029A00F012F9380000F064F950
:10815000029B002BDFD0300000F080F9DBE70378D2
:10816000032BD8D16288029909A800F0D6F8DEE77F
:10817000122B13D1029909A800F0B5F8021EEAD11A
:1081800027498B88002BC6D0887909A923780191CB
:1081900061780091310000F0EAF8BCE7002302AA00
:1081A00093833000617809AAFFF72AFFB3E71D4BDC
:1081B0000993F6E7042B02D09A1F012AABD8184A7C
:1081C000043B9B00995A0029A5D0D2189078310021
:1081D0003A0000F0AEF800289DD13B88042B03D074
:1081E00001213000FFF724FF012C04D1A8680028EA
:1081F00001D003F011FB280003F05EFA8020039BFE
:108200000002434018000DB0F0BD012800D182E704
:1082100001213000FFF70CFFEDE7C046E864FF1FC7
:10822000D864FF1F010017000B7803704B78437070
:10823000CB788A781B021343438070470A88030077
:1082400002700A88120A42700A88012A06D14A88F6
:1082500082704A88120AC27004207047022082424B
:10826000FBD14A8804309A704A88120ADA708A88E8
:108270001A718A88120A5A71EFE710B504000120BA
:1082800082420CD94B780A781B0213432380834225
:1082900006D1CB788A781B0213436380002010BD7F
:1082A000022BFBD1CB788A781B02134363804B7976
:1082B0000A791B021343A380F0E70B8803700B8835
:1082C0001B0A43704B8883704B881B0AC3708B88D2
:1082D00003718B881B0A4371CB888371CB881B0A7F
:1082E000C3710820704703000120082A14D14A787E
:1082F0000878120202431A80CA7888781202024370
:108300005A804A790879120202439A80CA79887998
:10831000120202430020DA80704710B504000120E9
:10832000022A05D100204B780A781B0213432380D0
:1083300010BDF8B5060010200F00150003F06CFC0E
:1083400004000120002C0ED0A0230C222900238041
:108350006780201D002D07D003F08EF9210030002A
:1083600003F092FC0020F8BD03F0B6F9F6E7F7B58C
:108370001E00009008AB142017001D78019103F037
:108380004BFC041E12D0A2230370019B4770438054
:10839000099B057146710C220830002B07D019008B
:1083A00003F06AF92100009803F06EFCF7BD09990B
:1083B00003F092F9F6E737B5041E0FD04388002B7F
:1083C0000CD00025C1881323007A1722019500954F
:1083D000FFF7CDFFFF2365806372257037BD000076
:1083E00010B50C4904004A88002A09D08B89002B5B
:1083F00005D00020CB8A0222834201D010BD012289
:1084000013000A20434300204032C854C818428059
:108410000472F3E7BA64FF1F0023438003707047C0
:10842000094B00211A0010B55C88002C06D01C797D
:10843000844203D10A234B43D01810BD01310A33C3
:108440000329F1D10020F8E7BA64FF1F10B504003A
:10845000407A03F0F1F9FF23637210BD70470430D6
:1084600010B580B203F0B8FA002803D004214942C5
:1084700003F0DAFB10BD000070B50025104CA068B9
:108480002580A581A580A84202D003F0C5F9A5608A
:1084900000250C4C0C4B606D1D80230058331D7063
:1084A000A84202D003F0B8F965650025606800288D
:1084B00001D003F0B1F9013508340A2DF6D170BDB1
:1084C0008065FF1F2465FF1F7465FF1F70B5041EC4
:1084D00009D1054D2880A881A880A868002802D06D
:1084E00003F09AF9AC6070BD8065FF1FF0B54B8852
:1084F00085B00193002343600A7905000F00022A2A
:1085000000D07BE0CA88032A17D98B685E78197877
:108510003602DC78D8790E4399781B7A24021B0244
:108520000C43034353495BBA0B80331D93421ED166
:10853000042C04D0631F022B0ED9012015E0019AF0
:108540004D4B1201D35A002B06D00198FFF7BEFF06
:108550004A4A1369013313610421B8682E812C80C3
:10856000494203F061FB6860002005B0F0BD434D57
:10857000042C06D0631F022B0FD9EB680133EB608C
:10858000DBE7019A3C4B1201D35A002B05D001982E
:10859000FFF79CFF2B6901332B61374B30000293AF
:1085A000019B029A1B010193002301998C468B5277
:1085B000130063449C8003939E81FFF750FF039B4D
:1085C000041E986016D00421B868494203F02CFBC1
:1085D000FA880100043A200003F04EF80199029A4B
:1085E000FB888A5A043B9B18029A8B522B680133F2
:1085F0002B60A2E7AB690133AB619EE71E4B029390
:10860000019B1E01029BF35A002B2DD002998C195D
:10861000A068002828D0012A26D1FA889B189BB28E
:108620007352A189994217D39B1AC018B96803F0F5
:1086300023F8029BA289F35A934200D07DE70022DF
:108640002B81A3882B80A3686B60029BF2520B4A9C
:1086500053680133536070E7084A936801339360AD
:108660000198FFF733FF68E7044A53690133536108
:10867000F6E7C046EA64FF1F8065FF1FF064FF1F36
:1086800070B5051E15D10B4C0B4B188023005833C9
:108690001870606D002802D003F0BEF865652500F3
:1086A00050356068002801D003F0B6F80834AC42B9
:1086B000F7D170BD2465FF1F7465FF1FF0B517006B
:1086C000A12285B0920001934243394B06001B68FA
:1086D0000C009B18D933FF331D78FDF741FF0430A0
:1086E000854204DD3000FDF73BFF0430C5B2BD42DA
:1086F00007D33A0000213000019B03F00DF805B0CC
:10870000F0BD2900380003F0E7F82300C6B250336B
:108710001E700393019B29006365380003F09CFAE7
:10872000CBB20293002B02D0039B01361E700026B1
:108730002300503303931B78B34204D8606D0028A4
:1087400031D10020DBE7029A2800002A04D0013B47
:108750001000B34200D02800F700E719387003F08A
:1087600043F8786000280ED03A78019902F084FF2F
:10877000019A3B780136D3180E4A0193D369F6B2B9
:108780000133D361D4E7039B18706065A74205D11C
:10879000084A1320D36A0133D362B0E7606803F05C
:1087A0003BF80834F2E703F037F800236365C8E7C5
:1087B0003409FF1FF064FF1FF7B50D000700042107
:1087C000686803F031FA2B89040003702B891B0AB7
:1087D00043702B8883702B881B0AC3702E89022557
:1087E0000436F6B2F42E15D81B4B9F4214D10C2040
:1087F00003F012FA1135011E0CD0902303708E3B4A
:108800000371043B4380154B8460C680187803F0E5
:108810003BFA00252800FEBD5C237B43104AD31899
:108820000093583301931B78002B0FD103003200C3
:1088300038000099FFF742FF019B05001B78002BD1
:10884000E8D13800009902F0DFFFE3E7054A072589
:10885000536A01335362DDE7FEFF0000E864FF1F47
:108860002465FF1FF064FF1FF0B587B0009017204C
:108870000F0016000193FFF7F2FD1325041E19D017
:108880000C98031E02D00199201D9847030AE3703B
:10889000052302AAA07004309081277000986670AA
:1088A00003A993800494FFF787FF051E02D02000E0
:1088B00002F0B2FF280007B0F0BD0000F0B587B0AD
:1088C0001F000CAB1B780391059301210DAB060033
:1088D0001C78049200F0D6F81425002821D020003E
:1088E000FFF77EFD0135041E1BD01149059B0A7858
:1088F00003700132D2B2131EC68001D101231A00C7
:108900000B7022713000049B03990097FFF7ACFFB6
:10891000051E09D1230021000648074A093303F048
:10892000D3F8280007B0F0BD002363802370F8E778
:10893000EC64FF1FB783001130750000F8B5050027
:108940000E00064C064F2368002B02D03100280091
:1089500098470434BC42F6D1F8BDC0469065FF1F6D
:10896000A465FF1F0123064A5B4253800023137155
:108970005362044A136053609360D360136170477D
:10898000A465FF1F9065FF1F0200002310B5064974
:108990009C000859002801D1625010BD0133052BFD
:1089A000F6D11320F9E7C0469065FF1F034A5388AC
:1089B000181A43425841404210407047A465FF1FB7
:1089C000F0B585B002930AAB1F780CAB1B88009002
:1089D00008000E0001920393FFF7E8FF0500112045
:1089E000002D1BD10E48FFF7E1FF04001520002CDD
:1089F00014D006220B99A771E01D02F03DFE019BE9
:108A000030002371029B29006371009B66802370F4
:108A1000039B6562E381FFF791FF280005B0F0BD7D
:108A2000FFFF000010B5FFF7C1FF04000220002C7B
:108A300012D060880121FFF781FF606A002801D011
:108A400002F032FE28220021200002F045FE012320
:108A500000205B426380207110BD000030B5074AE2
:108A6000074C5588010013780020A54204D05B1AFA
:108A700059424B415842104030BDC046A465FF1FCB
:108A8000FFFF0000084A10B501230C00904208D0F7
:108A9000FFF78CFF031E04D0037923405A1E934135
:108AA000DBB2180010BDC046FEFF0000024B187973
:108AB000431E9841C0B27047A465FF1F70B5040003
:108AC0000D001600FFF772FF002804D10D4B9C42E9
:108AD00000D0143070BD416A03790520002907D009
:108AE00012221A40102A02D10520002EF2D10F20A6
:108AF000DB06EFD5897E0C20A942894149424942D3
:108B00000840E7E7FEFF0000030010B5002800D191
:108B100010BD0348034A41889142F9D09847F7E7CE
:108B2000A465FF1FFFFF0000002330B5C45CCD5CCF
:108B30006C40D4540133102BF8D130BD0F230022E8
:108B400010B5C45C64002243CA54C25CD209013B24
:108B5000F7D210BD0200010010B52032103102F032
:108B60007BFD10BDF0B58BB003901020059317006E
:108B7000049102F0D9FD0090102002F0D5FD009B79
:108B800013240190002B05D000280CD11324009849
:108B900002F08AFD019B002B02D0180002F084FD38
:108BA00020000BB0F0BD102002F0BEFD060010202A
:108BB00002F0BAFD13240500002E00D1AEE000281B
:108BC00019D01022002102F087FD320029000398FD
:108BD00002F042FD041E0ED133787F2B51D83000B5
:108BE0000099FFF7ABFF009B1B787F2B53D80199AF
:108BF0000098FFF7A3FF300002F056FD002D02D0D1
:108C0000280002F051FD002CC1D1102002F08CFD93
:108C10000600102002F088FD0290002E7CD0002873
:108C200078D03A000F3223000125121105D00F33FE
:108C30003B4015B25A4253411BB26A1E1201002B2F
:108C400033D0049BD2B298180099029AFFF76CFFB8
:108C5000013D10220021300002F03EFDADB2049F24
:108C60002D017D19AF4242D0002C33D0300002F0EC
:108C70001BFD029B002B00D189E7180002F014FDB8
:108C800085E729003000FFF759FF28002549009AA1
:108C9000FFF74AFFA7E729000098FFF74FFF2800DA
:108CA0002049019AFFF740FFA5E70F210F400499E3
:108CB0008A18D9B28F4208D9D15C06A81954013359
:108CC000102BF6D1029A0199C0E7791A4842414126
:108CD000C901F2E73900300006AAFFF725FF32008C
:108CE000039806A902F0B8FC10370400BAE7002C7C
:108CF000BCD13000029906AAFFF716FF320006A980
:108D0000039802F0A9FC082204003100059802F043
:108D1000B3FCABE71324A9E71324AAE7002800D08B
:108D20006EE733E7D0BE0011F0B58BB00F00160030
:108D30000225009000283FD0002A3DD00B1DDBB259
:108D40001800029302F0F0FC1135041E34D0FDF738
:108D500047FD05003A000099201D02F0B5FCEBB27A
:108D60000393E3702B0CDBB22F0A00936370FFB206
:108D70002B0E2370A7700193FDF72CFD102201002C
:108D800006A802F0A1FC2100029A04AB06A8FFF796
:108D9000E9FE051E0DD1039B08223370009B04A938
:108DA000B370019B7770F370301D02F08DFCFDF7FE
:108DB0001DFD200002F078FC28000BB0F0BDF0B5DE
:108DC0008FB00D00149E039004920593002A03D1E6
:108DD000022420000FB0F0BD002EF9D00398FFF759
:108DE000E5FD1424071EF4D07278337812021A437A
:108DF000B3781B041343F27812061A43036A0192F4
:108E0000934201D30133E3D1002D03D03B790124F8
:108E10009B07DED50822002106A802F05DFC059B19
:108E200013240433DBB21800029302F07DFC051E0C
:108E3000CFD0059A0499043002F046FC0422310098
:108E4000280002F041FC3900102210310AA802F07B
:108E50003BFC2900029A06AB0AA8FFF783FE041E1A
:108E60000FD1082206A908A802F02EFC0822311D05
:108E700008A802F081FE012807D101990398FDF7A7
:108E8000C9FC280002F010FCA3E70124F9E7000068
:108E900070B51C4C05002368181E10D0002D14D18D
:108EA0001A78002A0CD1981C083202F0E5FB02F077
:108EB000EBFC0135002808D123681D70012070BD2E
:108EC0000A331800082202F0D7FB2368002BF5D0E4
:108ED000122002F0A1FE061E0DD0C12321680370EE
:108EE000457002311022023002F0C6FB23683100C7
:108EF000587802F0C9FE206802F0D6FB00232360F8
:108F0000DCE7C046CC65FF1FF8B504002020FDF764
:108F100055FB0D4EA700BB590500002B0DD00028B6
:108F20000BD0D878FF2809D108492A000C55F359ED
:108F300007480333611802F0C7FDF8BD290002F0AD
:108F4000DBFC0028F0D1F8E7E865FF1FD065FF1FC4
:108F500061A1001170B5064D84006359002B05D046
:108F6000D87802F069FCFF226359DA7070BDC04600
:108F7000E865FF1F70B506008CB00C0015000021DD
:108F80003022684602F0A8FB31001022684602F049
:108F90009BFB1D2021000322684402F095FB6846DC
:108FA000FFF7D8FD2D21040003222800694402F0B8
:108FB0008BFB20000CB070BDF0B50700160097B019
:108FC00001931CAB1D7830221EAB00910AA8002132
:108FD0001C7802F081FB102239000AA802F074FB11
:108FE0001022002102A802F077FB0722310002A81C
:108FF00002F06AFB072202AB9818631E9C4101999C
:1090000002F062FB02AB9C732B005A1E934102AA32
:10901000D3730021102206A802F05EFB06221D99E0
:1090200007A802F051FB1A2002ABC01806221F99B4
:1090300002F04AFB102200990EA802F045FB102214
:1090400002AB0EA908781C78013A6040D2B20870D1
:1090500001330131002AF5D10AA8FFF77BFD102268
:1090600012A904000EA802F007FB102206AB0EA9FD
:1090700008781D78013A6840D2B208700133013196
:10908000002AF5D10AA8FFF765FD044310222098B5
:10909000E4B212A902F018FB200017B0F0BD70B5C1
:1090A0000E0014008CB00100102268461D0002F072
:1090B0000BFB3100082204A802F006FB2100082265
:1090C00006A802F001FB6846FFF744FD04001022E9
:1090D000280008A902F0F8FA20000CB070BDF8B51D
:1090E00006000D0000243719AC4200D3F8BD02F091
:1090F000B3FC030A3B70631CDBB201379D4203D90A
:109100000234F054E4B2EEE71C00EDE773B506005C
:109110000C000225002819D0002917D0032101A82E
:10912000FFF7DDFF6B469A793F231A400133134363
:109130006A463000937101A92200FFF71BFF051E4C
:1091400004D10322E01C01A902F096FA280076BDA2
:1091500003785807DA08C00FD20080009B0710433D
:109160009B0F1843C0B2704707230B40C908C900C2
:109170000B4303707047000070B50400FFF7EAFE70
:10918000134DA4006359002B21D0186A002801D088
:1091900002F08AFA2B59986E002801D002F084FA66
:1091A0002B59D86E002801D002F07EFA2B59186F87
:1091B000002801D002F078FA2B59586F002801D00E
:1091C00002F072FA285902F06FFA00232B5170BD99
:1091D000E865FF1F0E4B8000C35870B50C00002BD4
:1091E0000FD09D68002D0CD02B78201D0B706B7854
:1091F0004B70A97CFFF7B8FF2B7E23726B69E3608D
:1092000070BD10220021200002F066FAF8E7C04687
:10921000E865FF1F014B18607047C046E465FF1FFB
:10922000074A03008000825810B5002A06D0D08873
:10923000984203D1012901D1FFF79EFF10BDC0461E
:10924000E865FF1FF0B5264E95B087000B93BB591C
:109250000500099112200A92002B31D0D888FFF71F
:10926000A5FB04001420002C2AD0280010A9FFF729
:10927000B1FFBB591E781D6A002E23D00895FDF75B
:10928000EFFA07000020FDF7F1FA0790A379E61D39
:10929000069310AD0CA9089800F0E2FA0EA9280078
:1092A00000F0D7FA0B9B0A990493069B0998029346
:1092B000079B0396019300970EAB0CAAFFF77CFE69
:1092C00015B0F0BDFDF7CCFA06903000FDF7CEFAF0
:1092D000E31DA779079310AB06000893DAE7C046B1
:1092E000E865FF1F30B50C4C85002A59030085B096
:1092F0000120002A0ED018006946FFF76BFF2B599A
:109300001A78D888054B002A00D1054B6A460721F8
:1093100000F0D9FB05B030BDE865FF1F5398001180
:109320006198001130B5094C8500295985B010228B
:109330006846253102F0A0F92A591121044BD08842
:109340006A4600F0C0FB05B030BDC046E865FF1FAF
:10935000FD98001130B5094C8500295985B01022BF
:109360006846353102F088F92A591121044BD0881A
:109370006A4600F0A8FB05B030BDC046E865FF1F97
:109380003B990011F7B54D4F86001020F4590D00A0
:1093900002F0CAF9F3592062186A132200286CD02F
:1093A000033A29009C6802F067F9F3591A78019290
:1093B000002A58D11E6A227D317B944651400122F9
:1093C000019F114201D167461740217D91433943E6
:1093D0002175377B4F40BC4660460027800701D48B
:1093E0004F081740012102208F40227D82433A43DB
:1093F0002275377B5740BC4660460027400701D4A2
:1094000097080F400420227DBF0082433A43227513
:10941000627D002794466046727B42400A4201D139
:1094200067460F400121627D8A433A436275777B2C
:109430005740BC4660460027800701D457080F40BC
:109440000220627D7F00824317436775767B00228E
:109450007E40760701D4BA080A400426617D920056
:10946000B1430A4362756A78002A08D06278002AFC
:1094700005D005220533DA7700221000FEBD042254
:109480002979114205D1A17C114202D10533033A59
:10949000F1E7019A21782C78002A02D10A002100F4
:1094A000140018220429E8D8042CE6D805206043CB
:1094B000034A05331218525CDDE7C046E865FF1F1A
:1094C000E0BE001110B50A001121024B00F0FBFABA
:1094D00010BDC046979900110B0030B587B001ADA3
:1094E0002B806B4604001100981D082202F0C4F87E
:1094F0002A000B212000024B00F0E5FA07B030BD36
:10950000BF99001110B50A001121024B00F0DBFADF
:1095100010BDC046139A001113B50B0011006A4626
:1095200013706B4604000622581C02F0A5F86A4628
:1095300008212000014B00F0C6FA13BD339A001138
:1095400010B50A001121024B00F0BDFA10BDC04653
:10955000839A00117FB505000B4BAA00D458080070
:10956000002C0FD0666F237FE28821780396266F48
:109570000296E66E0196A46E0094FDF709FC2800A1
:10958000FFF7FAFD7FBDC046E865FF1F10B5172144
:10959000FFF7E0FF10BD000070B50A000D00064B9C
:1095A0000221040000F08FFA060029782000FFF75E
:1095B000D1FF300070BDC0466399001170B586B010
:1095C00000236A461370836804001D78681E0A2809
:1095D00059D801A902F010FB060633373B3F434739
:1095E0004B4F5300180000F042F9062312284BD0CD
:1095F00000281BD16088FFF7D9F90823002813D071
:109600004279002A47D1264B1A78072312070BD537
:10961000244B1A680723002A06D01668002E03D0B0
:10962000290001AAB04703006A4613706B461B78F5
:109630006088002B2AD1FFF767FC06B070BD1800C8
:1096400000F06CF9D4E7180000F087F9D0E71800B3
:1096500000F093F9CCE7180000F0ADF9C8E7180066
:1096600000F0C3F9C4E7180000F0F6F9C0E71800ED
:1096700000F0F6F9BCE7180000F013FAB8E718009C
:1096800000F013FAB4E707236A461370694660884E
:10969000FFF782FFD1E70523012AC5D1024BB8E7C6
:1096A0007564FF1FE065FF1FE465FF1FF8B52C4FD1
:1096B0008600F35904000D00002B40D0DA88824266
:1096C0003DD15A78062A33D11A78002A2ED00120AB
:1096D00099681A6A097D014206D0157B054203D0BC
:1096E00007225A700120F8BD0220014204D0157BE8
:1096F000054201D00922F4E70420014204D0127B84
:10970000024201D00B22ECE7164B1B68002BE9D07C
:109710005B68002BE6D020009847BB5900215B789E
:10972000122BDFD12000FFF715FFDBE70E4BECE734
:10973000112A04D1002900D032252900F2E7002D9A
:1097400008D12000FFF732F9002803D01023027956
:109750001343037121002800FDF798FAC2E7C046C1
:10976000E865FF1FE065FF1FE465FF1F70B50E4E43
:109770008500AB590400002B13D01B78002B11D1AE
:109780000A4B1B68002B04D05B68002B01D0200023
:10979000984773595B78122B03D100212000FFF703
:1097A000D9FE70BD024BECE7E865FF1FE465FF1FC3
:1097B000E065FF1F094B8000C3581020002B0CD020
:1097C0001A6A002A09D09B68002B06D0127A1B7EE9
:1097D000101C9A4200D9181CC0B27047E865FF1FE0
:1097E00070B503000D0014000220002A30D00029BB
:1097F0002ED013700B78081D53704B789370FFF7C1
:10980000A7FCE070012002212B7A23716B7B0340BF
:1098100063716A7B0A401343042263716E7B1640B6
:10982000334363716E7BF608F600334363712B7B21
:109830000340A371287B014000200B43A371297BC7
:109840000A401343A3712A7BD208D2001343A371A9
:1098500070BD10B50A0001000120FFF7C1FF10BD67
:1098600010B50A0001000220FFF7BAFF10BD70B565
:1098700006000C000220002E30D000292ED0737874
:10988000201D0B70B3784B70F178FFF76DFC01224F
:109890003579257271794B100800134093401040C0
:1098A0000343881010408000C9080343C9000B43DC
:1098B0006373B1794B100800134093401040034389
:1098C000881002409200C9081343C9000B432120AD
:1098D0002373FCF773FE854201D2122070BD222053
:1098E000257AFCF76BFE8542F7D823781820042BE5
:1098F000F4D86378012BF1D80020EFE7030010B50E
:109900000220002909D0002B07D00322481C0A702E
:1099100019000D3201F0B0FE002010BD030002223C
:10992000080010B5002B06D0002904D00E32591CB7
:1099300001F0A2FE0022100010BD030010B50220AD
:10994000002909D0002B07D00422481C0A701900F6
:109950000C3201F091FE002010BD10B5FFF7DEFFC4
:1099600010BD03000220002906D0002B04D00522E0
:1099700000200A701B784B70704703000220002BF8
:1099800008D0002906D05B7800200B70013B082B23
:1099900000D918307047030010B50220002909D003
:1099A000002B07D00622481C0A7019000A3201F069
:1099B00063FE002010BD10B5FFF7B0FF10BD020020
:1099C0000B00022010B500290ED0002A0CD0072170
:1099D0001970118859701188090A99701118082294
:1099E000D81C01F049FE002010BD03000A0002202F
:1099F00010B5002B0CD000290AD0997858780902AC
:109A000001431180901CD91C082201F035FE002072
:109A100010BD030010B50220002909D0002B07D08B
:109A20000822481C0A701900921801F025FE002037
:109A300010BD02000B00022010B500290BD0002A37
:109A400009D009211970117818185970511C062273
:109A500001F012FE002010BD10B5FFF75FFF10BD32
:109A600002000B00022010B5002A09D0002907D0FF
:109A70005178197011180622581C01F0FDFD0020C4
:109A800010BD030010B50220002909D0002B07D01B
:109A90000A22481C0A701900063201F0EDFD002070
:109AA00010BD10B5FFF73AFF10BD02000B000220F9
:109AB00010B5002A06D0002904D018005178FFF70D
:109AC00053FB002010BDF0B585B017001E006A469C
:109AD00006230500080091819380FEF7C0FC132443
:109AE000011E02900CD03800B047041E05D128009A
:109AF00001A9FEF76FFA041E02D0029801F08CFE55
:109B00002800FFF701FA200005B0F0BDF0B5040011
:109B10008BB0019115000021102202A801F0DCFD9C
:109B2000334EA700B85900283CD0C388A34239D18E
:109B30000378002B36D14278062A18D102000100A2
:109B4000553235310C3006ABFFF7A9FA002829D180
:109B50002000FFF72FFE020006A902A801F08CFDED
:109B6000200002A901F090FD01200BB0F0BD816E34
:109B7000002917D00B8A112A28D19D420ED10198B5
:109B80001231093A01F0F8FF012807D1BB59200032
:109B90009D6EFFF70FFE29000200DEE73221200054
:109BA000FFF7D8FC2000FEF701FF061E1BD0416A1C
:109BB000002918D00B8AAB4215D108220198123126
:109BC00001F0DAFF01280ED1716A0AE09D42E9D165
:109BD00008220198123101F0CFFF0128E2D1BB59D0
:109BE000996E8A7EB9E7200001F096FEBCE7C04678
:109BF000E865FF1FF0B56B4D87007E5985B033785F
:109C000002900393002B00D087E0B368346A01937D
:109C10007078062817D101221B7D134202D0217BC8
:109C2000114218D10222134202D0217B114251D19C
:109C30000422134203D0237B134200D08BE0019B0C
:109C40005A7DEB5991E007380428F8D801F0D4FF89
:109C5000032E42678300B36E002B03D11C2001F05A
:109C600063FDB066EB599C6E002C1CD010220021C5
:109C7000200001F031FD0298FFF79CFD010020005B
:109C8000FFF72DFA01F0E8FE2082200008211230B3
:109C9000FFF725FA0298FFF78DFDA076EB5921001A
:109CA000D888FFF70FFC0822EB591CE0B36E002B9D
:109CB00005D01A00198AF0881232FFF70DFC022233
:109CC000019B197DEB5911423DD0207B10423AD0C7
:109CD000073208E0F488FCF7DBFD01002000FFF705
:109CE00011FC0A22EB595A70029B9C002A595378A6
:109CF000073B042B11D8D088FEF758FE00284ED021
:109D0000C3895A08D2182849029B0298CB542B5970
:109D100041180433254801F0D7FE05B0F0BDFCF72B
:109D20009FFD03000120834201D100200393EB59E2
:109D3000DE88FCF79BFD039902003000FFF7ECFB87
:109D4000019AEB59117D042211420CD0217B114262
:109D500009D00B22C7E7F688FCF73CFD0100300074
:109D6000FFF7EEFB6BE7019A527D01210A4204D016
:109D7000607B084201D00C22B5E702210A4204D0E0
:109D8000607B084201D00E22ADE704210A4204D0D4
:109D9000627B0A4201D01022A5E71222A3E7FA2231
:109DA0005200B0E7E865FF1FEC65FF1F6BA10011D3
:109DB00010B5064B1A780423100018401A4200D040
:109DC0000348FFF727FA002010BDC0467564FF1F47
:109DD0002043FF1F70B50400FFF7D4FA051E43D1DE
:109DE0002000FFF77FFA234EA400A0598268937CDD
:109DF000DB0708D50321036A1B790B40012B02D135
:109E0000017F0B430377431DD97F8B1E022B0DD897
:109E1000022900D00121C088FCF790FF04213359AA
:109E20001A7F59700A431A77280070BD01290CD196
:109E300002231022437000210C3001F04DFC3059F8
:109E400010213530FFF74BF9EEE70529ECD102235D
:109E5000D118437010220C3001F00EFC042332594B
:109E6000117F0B431377EAE708251828DCD1053D5D
:109E7000DAE7C046E865FF1FF0B58BB0059143886F
:109E80007E4F9E00F45915000493002C15D1012932
:109E900002D000200BB0F0BD101D57781678FFF7E8
:109EA00057F9EB68320002932B7A049901930090E2
:109EB0003B002000FCF70CFFEBE7E388049A934299
:109EC00001D00820E6E72378012B00D1D4E0059BE0
:109ED000581E092800D9CFE001F08EFE05CE0A29D0
:109EE000CC506C859AB229000498FFF773FFD1E734
:109EF000200029001022453001F0BEFBB9594B78F3
:109F0000042B02D1013B4B70C3E70B000A00253341
:109F100035320C310498FFF795F90498FFF702FAEF
:109F20000522431E9841BB59C0005A70B2E7200079
:109F300029001022553001F09FFB049B4F4C9D00DF
:109F4000295904980A0006AB55320C31FFF77AF90B
:109F500029591022453106A801F00EFE012808D12A
:109F60000498FFF7F7F90590002804D106222B5931
:109F70005A7005988EE708230593FAE763780C2B4F
:109F80007AD1E36E002B03D11C2001F0CDFBE066FB
:109F9000BB59D86E00286FD01022290001F06CFB4D
:109FA000BB590498DC6EFFF705FC0D22A076BB5967
:109FB0005A706EE7E06E00285ED063780D2B5BD19F
:109FC0002B8808220382A91C123001F055FBBB59D3
:109FD0009A68517D0222114226D0186A407B1042B5
:109FE00022D00C32E4E763780E2B45D1236F002B8F
:109FF00003D1162001F098FB2067BB59186F002889
:10A0000003D01022290001F037FB0F22BB59CFE704
:10A0100063780F2B30D1206F0622691C103001F0BD
:10A020002BFBBB599A68517D0422114203D0196A57
:10A03000497B1142D5D100210498FFF78BFA28E71C
:10A04000636F002B0DD0BB59586F0028F3D010223E
:10A05000290001F011FB0122BB5952425B6F1A61CA
:10A06000E9E7142001F060FBBB5960675B6F002BD0
:10A07000E9D126E72978DFE707200BE7E865FF1F2E
:10A0800010B5064C207001F07FFC06212078FDF70A
:10A0900091FF0348FEF778FC10BDC046FB65FF1F2B
:10A0A0002192001100200BB270B50D00834216DA28
:10A0B000264B187801F0E8FC041E0DD00378922B93
:10A0C0000ED0A02B37D0224B1878FF283AD0210091
:10A0D00001F0DAFD002835D180200002684070BD13
:10A0E00043780E2B0BD03E2BEDD18378052B12D06D
:10A0F000082BE8D181798088FFF7D8FA08E0154B62
:10A1000082889A42DFD183681878591CFEF7C0FE16
:10A11000002817D1D7E7104B1B785B0712D50F4BE0
:10A120001B68002B0ED09B68002B0BD0C289811DB1
:10A1300080889847ECE7FFF741FAA068002801D033
:10A1400001F06AFB200001F0B7FAC5E7FB65FF1FCD
:10A150001943FF1F182000007564FF1FE465FF1FEF
:10A1600010B50078FFF712FA10BD10B50078FFF7B0
:10A17000FDFA10BD0C234343084A10B59B185A68DA
:10A18000002A03D0012901D1904710BD9B68002B04
:10A19000FBD00029F9D19847F7E7C0461866FF1FA2
:10A1A00001238340094A10B5946B1C439463506BA0
:10A1B00098435063D46B20009843012901D12000BB
:10A1C0001843D063116B0B43136310BD0080004034
:10A1D000F0B500240127154B85B0DA6B144E0392BD
:10A1E0001A6C0192DA64019BE3403B4217D0039D55
:10A1F000E5403D400295E5B202992800FFF7BAFF1D
:10A20000316A736A002908D03900002B01D0029905
:10A2100079402800FFF7C4FF01E0002BF9D1013499
:10A220000C36172CDFD105B0F0BDC04600800040D1
:10A23000FC65FF1F064B01215A68C2400A4204D048
:10A240001B68C3401800084070471B6DF9E7C04603
:10A25000008000400122064B8240002903D0D968CB
:10A260000A43DA607047D9689143D960FAE7C0467B
:10A270000038004030B5032444430F4BE25C1B1907
:10A280009C785D7801232D1B0135AB40013BA34039
:10A29000A140DB430C00122807D80849920052184D
:10A2A000116819402143116030BD054A11680B4007
:10A2B00023431360F8E7C04627BF001108F00040B1
:10A2C00014F00040C21F70B5D4B20623092C0BD87D
:10A2D0000125084C9540002908D00021FFF7CAFF4E
:10A2E00023682B4323600023180070BD2368AB4311
:10A2F000F8E7C04600380040214BF0B51B185B78EA
:10A30000022B21D1032444431E4A1F4EA35C121981
:10A310009478012215008540B76B013CE4B23D43BF
:10A32000A240B563194C122815D89B0000290CD106
:10A3300017495B1899680A439A600123205C154A03
:10A34000834011680B431360F0BD11495B18996895
:10A3500091439960F1E70E4B00290DD159690A43E9
:10A360005A61225C1328E8D00123203A93400A491D
:10A37000086803430B60E7E7596991435961F0E7C7
:10A38000FC65FF1F27BF0011008000406CBF00115B
:10A3900000F00040A0F00040A4F00040F8B5002418
:10A3A0001B4E1C4D1C4B1B5D012B1FD1194A926982
:10A3B000E2401A420BD00122B25693402200143AD6
:10A3C000D2B2022A09D815494A6913434B610134B4
:10A3D00002360C35172CE5D1F8BD0022B2560F49D4
:10A3E0009200521891680B439360F0E7022BEED174
:10A3F000E7B23800FFF71EFF01235840C1B2380012
:10A40000FFF77AFF3800FFF715FF6877DFE7C046F0
:10A41000F9BE0011FC65FF1FFD65FF1F00F0004045
:10A42000012202388240054B002903D059690A43B2
:10A430005A617047596991435961FAE70038004001
:10A44000F8B50E0001210F008740114A0400D368BF
:10A45000FD43BB43D360831E8B4201D8FFF7E0FF6F
:10A4600000212000FFF72EFF0A4A0B4B5168012EF6
:10A4700005D139431B1951605E700020F8BD294099
:10A48000516002221C1962709A6915409D61F4E7BF
:10A490000038004000800040FC65FF1F012210B51D
:10A4A0008240074B002906D019680A431A6001212F
:10A4B000FFF7C6FF10BD196891431960F7E7C04662
:10A4C000008000400C2370B5002543430A4A290050
:10A4D0009B181D70094B04001B185D70FFF7B0FF3F
:10A4E0000123A340064928000A681A430A60054967
:10A4F0000A689A430A6070BD1866FF1FFC65FF1F5B
:10A50000348000403080004070B504000E00FF2809
:10A5100013D003250540FFF7D5FF084AA3089B0089
:10A520009B183F22ED00AA40AE40196820009143DD
:10A53000314319600121FFF78DFE70BD18380040CE
:10A54000F8B50C244443134B0500E4186368002B52
:10A5500003D1A3681220002B1AD0022201270E4B30
:10A5600000215B195A7028002770FFF769FF6368A4
:10A570001E1E08D0A3683E00002B04D02800FFF761
:10A5800059FE4640F6B228003100FFF709FE0020D0
:10A59000F8BDC0461866FF1FFC65FF1FF7B5C42055
:10A5A000FF222B4B80001958002491433F3A0A4365
:10A5B0001A508022274F5202274E1A60274B1D5DEA
:10A5C000002D21D0A31E012B03D80121E0B2FFF7FB
:10A5D00027FF012D18D11F4B9B69E3402B4213D05D
:10A5E000E3B218000193FFF725FE01000198FFF781
:10A5F00055FFE3B2143B022B1DD801217156184AB6
:10A600008D405369AB4353613B7F002B0DD0E5B2C6
:10A610002800FFF795FF2800FFF70CFE7B7F010065
:10A62000834202D02800FFF7A5FD01340C37023623
:10A63000172CC3D1F7BD012100237156F3568D406D
:10A64000074A9B009B189A68AA439A60DCE7C046B9
:10A6500000E100E0FC65FF1FF9BE0011FD65FF1F72
:10A6600000F0004010B501210400FFF7E9FE0123CE
:10A67000044A002011194B70A34091690B43936168
:10A6800010BDC046FC65FF1F70B50E00150004002C
:10A69000FFF718FF0C236343094A20009B189D60B5
:10A6A0005E60FFF74DFFF021064B074A8900051E4B
:10A6B0005A5002D02000FFF705FF280070BDC046A9
:10A6C0001866FF1F0000FF1FD1A1001170B5134DC8
:10A6D00007202C78002C1FD198222100520028003E
:10A6E00001F062FA0123C420FF222B700C4B800082
:10A6F0001C635C630B4B1C605C600B4B19589143F3
:10A700003F3A0A431A50802252021A600D20074A2B
:10A71000074901F0D9F8200070BDC046FC65FF1F55
:10A7200000800040A0F0004000E100E09DA5001185
:10A730009DA30011030010B50620072B09D8054A78
:10A74000137001F099FAD7210020034B034A8900C6
:10A750005A5010BD4843FF1F0000FF1F8D1BFF1FF5
:10A7600070B51D0002240C2910D8094ACA40D2072E
:10A770000CD5FBF72FFF041E08D1059A0499280079
:10A78000FBF744FFFCF7B2FDFFF712FB200070BDA2
:10A790001210000030B50D7802232C009C431842A3
:10A7A00001D02B431C0008252300AB43284201D0D5
:10A7B0002B00234320241D00A543204201D01C432D
:10A7C00025002A230D70184204D011781E3B0B433C
:10A7D000137030BD0028FCD10C2113788B43F7E7B0
:10A7E000F8B51D0006AB1B88140007AA0E000B204D
:10A7F0001778002B27D10A78022A49D14A68507865
:10A8000011780002244A08438018042840D801F037
:10A81000F3F903121D1B2300F06801F0F5F8021C88
:10A82000C0B2B84200D93A1CD2B22000F1682A80E6
:10A8300000F022FF06E00222F3681B882A802370C2
:10A840001B0A63700020F8BD0622EEE701232B806F
:10A85000F3681B782370F5E7F368002B16D0082205
:10A860002A801A8822701A88120A62705A88A27086
:10A870005A88120AE2709A8822719A88120A6271C2
:10A88000DA88A271DB881B0AE371DBE72B80D9E74A
:10A8900001202B80D7E7C04600D6FFFFF7B5160092
:10A8A0000A781D0008AB1F880C000123022A18D16A
:10A8B0004A685078117800022B4A08438018032810
:10A8C0000FD801F099F902254439E06801F09CF8AD
:10A8D000C0B20723B84204D37B190193152B02DDC4
:10A8E0000D231800FEBDE0682A003100C01900F0F9
:10A8F000C3FE6B4600209B88E268D0541B4B1B684C
:10A90000834203D01B68834200D098470023E8E7C6
:10A910000B23002FE5D1022DE2D1737832781B0290
:10A920001343E2681380114B1B68002BEED01B68A9
:10A93000002BEBD00120E8E70B23002FD1D1062D0F
:10A94000CED12A003100E06800F096FEDEE70B234E
:10A95000002FC6D1012DC3D132787533012AC0D85A
:10A96000E3681A70D2E7C04600D6FFFF0868FF1FF1
:10A9700070B50C001500072837D801F03DF9041414
:10A9800036361B36242E182015290BD8184E1622C1
:10A990000021300000F0A0FE22002900300000F06D
:10A9A0006BFE002070BD18200229FBD11288114BCC
:10A9B0001A80F6E718200829F4D10A000E48290069
:10A9C00001F09AF8EDE718200129EBD10B4B107834
:10A9D0000B49DA69FFF7DEFEE3E718200129E1D130
:10A9E000064B10780749DA6BF4E70220DAE7C04635
:10A9F000F067FF1FC643FF1FBC43FF1F4C43FF1FF1
:10AA00007443FF1F9443FF1F030010B50020DB07B2
:10AA100004D50721024A034800F08CF810BDC04657
:10AA200084BF00114C43FF1F054A03001068002833
:10AA300003D082889A4201D1806870470068F6E7A7
:10AA4000006AFF1F0A88030008009A4204D08A881F
:10AA500004309A4200D0002070470000F8B5F2227E
:10AA600000230D4F0D4E7968050042433370994223
:10AA700000D07B600A4C0021200000F02DFE002356
:10AA80001A007C60AB4202D100203370F8BD013364
:10AA90002280DBB2F234F5E7F86AFF1FF66AFF1F87
:10AAA000046AFF1F73B56B460190060068461500E7
:10AAB0001980FCF74DFF041E11D1002D0FD07689AF
:10AAC000002E11D00C2000F02FFE00280ED0084AD6
:10AAD0000460136886808560002B02D1106020001E
:10AAE00076BD1A001B68F7E70224F8E71324F6E79F
:10AAF000006AFF1F012100220A4B10B549420A4C8F
:10AB0000198099809A719A70084B207001201980E1
:10AB10005A60FFF7A3FF2078FCF778FF0448FDF7A1
:10AB200033FF10BD1068FF1F006BFF1FF86AFF1F87
:10AB3000E1AB0011022310B5002802D0FFF7B2FFED
:10AB40000300180010BD0000030010B50020DB0753
:10AB500004D50421024A0348FFF7A4FF10BDC046F4
:10AB600098BF0011CC43FF1FF0B50E2687B00393AA
:10AB70000CAB1F8802ABF6180500080031000292EA
:10AB8000FDF768F804000120002C0FD03088FFF793
:10AB90004BFF03000E20002B08D05E68002E05D06E
:10ABA00021002800039B029A0097B04707B0F0BD30
:10ABB0000A4B10B5984207D10122002352420A8065
:10ABC0008B708A808B7110BDFFF73CFF0028FAD094
:10ABD00001235B42038000238370F4E7FFFF000042
:10ABE000F8B5050001290AD1134E00243388F22755
:10ABF000AB4219D028001149FFF7DAFF06E002291D
:10AC000004D10139FDF73EFF0028EDD0F8BD3B002F
:10AC100063437268D018D35A002B09D03A00002140
:10AC200000F05AFD0134E4B2054B1B78A342EED884
:10AC300001235B423380DDE7F86AFF1F1068FF1FC6
:10AC4000F66AFF1F10B5FFF7FDFE030000208342E8
:10AC500000D0987810BD0000F0B589B01C000EAB94
:10AC600080CB03901E8810AB1B78049202930B7A62
:10AC70000D00DB0616D42B780593022B24D0049804
:10AC8000FFF7D2FE002812D003689C46002B0ED09E
:10AC9000029B2200019329003B0064460398009622
:10ACA000A04705E00498FFF7BFFE002802D10E2060
:10ACB00009B0F0BD8368002BF9D00A22290003985F
:10ACC00098470028D7D0F3E76B6858781A786B4B11
:10ACD000000210439842D2D8043B984210D2684BED
:10ACE000984242D015D8674BC0180128C7D80B200E
:10ACF000002EDDD1EB681A7859683A80200028E0F0
:10AD0000614BC018032800D979E000F075FF846A10
:10AD1000789E5E4B9842B2D10B20002EC8D1012301
:10AD20003B80EB6831001B7823706889013080B26A
:10AD3000FCF790FF3A88031E0ED0017802328A1881
:10AD40003A80428962704289120AA2705968027878
:10AD5000E01C00F091FC06E004323A80310004224D
:10AD6000601C00F0B9FC0020A2E70B20002E9FD150
:10AD7000EB6807A91E8804233B80330A3000267045
:10AD80006370FCF767FF051E28D004AB9A890E2379
:10AD900004A95B183E49C668FCF7D0FF00280BD118
:10ADA0002B783C486A680599FBF786FB002803D19D
:10ADB000012304AA5B42D3813278022A06D171684A
:10ADC000201D00F059FC3B8802333B800E2304AA6F
:10ADD0009B181B88A3701B0AE370C4E704ABDE81D9
:10ADE000F4E70B20002E00D062E7E9680398FFF734
:10ADF00029FF02233B802070000A6070B3E70B201C
:10AE0000002E00D054E70222EB681B883A802370A2
:10AE10001B0A6370A7E7E86800F0F6FDC2B2030002
:10AE20000720B24200D243E70DD00299DBB271187D
:10AE3000994202DB921BD3B20293029BE9681A008B
:10AE40003B8089195AE70023F6E70B20002E00D03B
:10AE50002EE70722EB683A801A7822705A786270DF
:10AE60005A88A2705A88120AE2701A792271DA8816
:10AE70006271DB881B0AA37175E7C04604290000D4
:10AE80000228000000D8FFFFFFD6FFFF03280000C4
:10AE9000FFFF0000C8BE0011F0B58DB06B4600206A
:10AEA000089120229B5E83423DDAA64B187800F081
:10AEB000EBFD071E32D00378B02B2CD1007902387D
:10AEC00016281FD800F050FD17001E001E001E009F
:10AED00031001E0096001E001D011E0052011E00C2
:10AEE00073011E00CD011E0050021E001E001E0038
:10AEF0008E021E00E302944B94491B8878880B80D5
:10AF0000FBF71AF83800FCF79BFF914B1B68002BEE
:10AF100001D038009847380000F0CEFB8020089B15
:10AF20000002434018000DB0F0BDEE22002187481A
:10AF300000F0D2FB0BAA3B7B7989388900923A005A
:10AF40000D32FCF79FFD0400804B1B78002C3FD195
:10AF500046E0804B788805937F4B4100CB5A0BAE7F
:10AF6000073BDBB232880293002301937B4B210025
:10AF700006930093059BFFF76FFE744D002810D1D8
:10AF8000069B3A8A1B889A420BD1380005991230E9
:10AF900000F0F2FD002804D02B7862899B00EB18AA
:10AFA0005A80162306A81B18328820007989FCF7DE
:10AFB000C5FE2B7804009A00AA1851880029C3D036
:10AFC0000133DBB22B70002807D006A9C98A918013
:10AFD000634A12889A42BCD802E00121494291801A
:10AFE000002B04D059497888FAF7DAFF8AE73E89BE
:10AFF0000A2479E000253E89574B06937B88069A00
:10B000005B009B5A033B9D4202DB002DF0D05BE0CE
:10B01000162206A812183B7B798900923A0030006C
:10B020000D32FCF72FFD0590002858D04689017A93
:10B030007888FCF7F1FC041E44D1464B78880793CE
:10B04000069B4100C95A454B0439C9B206AAD28AA7
:10B0500006930291019400930599079BFFF7FCFD6D
:10B06000041E2FD1069B39491A88931C002D26D126
:10B070004B807988384B4900CB5A5119033B8B429E
:10B0800020DD059B31485B8941190B71A91C0135F5
:10B09000C9B2EDB2059145191B0A2B71059B2D49CB
:10B0A0000433181800F0E8FA2C4B059A1B88D318C3
:10B0B000DDB22C4B9E4205D00136B6B29CE74988E2
:10B0C0009942D6D0002D0CD0204C2800618800F089
:10B0D000B3FA207021007888FAF772FF12E7059C16
:10B0E000F0E7002C00D183E77B78142B00D109E72F
:10B0F00016493B794E800B700C717888FAF712FF75
:10B1000000E7162406ABE41821003889FCF7A2FDFD
:10B11000011E00D1B7E1788822880F4C45002C5BD6
:10B120000A4D013CE4B2029400240F4B01940095B7
:10B13000FFF792FD041E00D014E129007888FAF789
:10B140004FFFDFE6006BFF1FB842FF1F1868FF1FAD
:10B150000C68FF1F0C69FF1F4864FF1FFC69FF1F7D
:10B16000B642FF1FFFFF00001A68FF1F162406AB40
:10B17000E41821003889FCF76DFD011E00D182E141
:10B1800078882288AE4C45002C5BAE4D013CE4B281
:10B1900002947C89AC4B01940095FFF75DFD041E81
:10B1A00000D0DFE029007888FAF724FFAAE600251E
:10B1B000A44B1D803B00F6331B78A24A7888079287
:10B1C000AB4208D99E4B12880693069943005B5AFE
:10B1D000013B9A4203DB0799FAF716FF92E6162421
:10B1E0006B00FB18059306ABE418059B210018893A
:10B1F000FCF730FD011E03D1059B01241E8973E776
:10B200007888924B2288069C099343001B5B904EE2
:10B21000013BDBB20293002300960193099BFFF7E9
:10B220001BFD041E02D0059B1E895DE77B88069AE4
:10B230005B009B5A079A108832881218934202DCEE
:10B240001B1A013B33807F4C023032880999001968
:10B2500000F012FA2388328801359B182380EDB262
:10B26000A8E70BAA3B7B7989388900923A000D3216
:10B27000FCF708FC00250590059B002B04D10A244F
:10B28000002D00D16EE060E0059B7888197AFCF70C
:10B29000C3FB0100041E63D1694C6C4B7888069493
:10B2A0000993069B4400E45A694B063CE4B20BAE9A
:10B2B000328807930294019100930599099BFFF747
:10B2C000CBFC041E4CD1079B5E491B881A1D002D28
:10B2D00030D14A80059B5B4C5A8963191A716B1CEB
:10B2E0009BB2E318120A1A71162306A832881B189B
:10B2F00079890598FCF722FDFF21AA1C2E1D033534
:10B300000B00059092B2B6B2ADB2002803D006ABE6
:10B31000DB8AD9B21B0AA218651911712B714C4D29
:10B32000301D2A884949201800F0A6F92B88F61804
:10B33000B5B2A1E74988914207D17A8806995200AF
:10B34000525AEB18053A9A42C4DC3E4C28006188F8
:10B3500000F0C2FA207021007888FAF75FFED1E58C
:10B36000002DF2D13E89BFE6162606ABF618310055
:10B370003889FCF76FFC3D000400FA3500282DD019
:10B38000037A9B060CD400227B8939897888009245
:10B390003A000C32FFF7E8FB041E10D03E8915E09E
:10B3A0003088FFF741FB00281AD08368002B17D0A4
:10B3B0002100122278889847041EE4D0EEE72B780B
:10B3C000002B02D17888FAF739FE00262B78002B63
:10B3D00000D097E5002C00D194E585E60124DDE757
:10B3E0000E24DBE7162506ABED1829003889FCF79B
:10B3F00031FC041E47D0037A9B0611D4154A7B8882
:10B400001188994203D01448814207D11380134B0D
:10B41000F2261D780023D9B2A94221D30924A1E73D
:10B420002888FFF701FB00282FD08368002B2CD041
:10B430002100122278889847041EDFD092E7C04688
:10B440004864FF1F1868FF1F1A68FF1F0C69FF1F61
:10B45000FC69FF1FF86AFF1FFFFF0000F66AFF1F6D
:10B4600031005943546801336018615A0029D2D120
:10B470003C0008342100F22200F0FEF82100788818
:10B48000FAF7E4FD3EE501246CE70E246AE71D4B64
:10B490001A887B889A4231D07888FAF7E1FD31E545
:10B4A000F223059851684343CD18C95A00291FD08B
:10B4B0003B7A012B0BD16C88AB887888AA1D00944D
:10B4C000FFF752FB041E02D000233B722E88F222AB
:10B4D0000021280000F000F900232B80059B013398
:10B4E000DBB20593084B05991B78064A8B42D7D8E7
:10B4F00001235B421380002CCED0F5E500263400FA
:10B500000596EFE7F86AFF1FF66AFF1F70B50400A3
:10B510000E001500FFF796FA031E08D1310005480A
:10B52000FFF790FA03001120002B02D01C800020AE
:10B530009D7070BDFFFF0000F8B50B4F06003B7813
:10B540000D001400FF2B0ED00A2000F065FB011E39
:10B5500009D0B1230380002346800371C580048194
:10B56000387800F091FBF8BD0D44FF1FF7B50F00D0
:10B5700008A90600088809A90B240988002821D1F8
:10B580000234022B1ED1557813782D021D432B0057
:10B590008B4301937334002B14D1FB6830001900E6
:10B5A0000093FFF74FFB019C85420BD02A0030002F
:10B5B0000099FFF7ABFF041E04D12A0030007989FF
:10B5C000FFF7BAFF2000FEBDF0B50E7885B00390FE
:10B5D0000AA805880120022E0DD14C6827786478CE
:10B5E00024023C43054FBC4205D10398DBB20196CF
:10B5F0000095FFF7BBFF05B0F0BDC0460229000073
:10B60000034B10B51B68002B00D09847FEE7C046DF
:10B61000046BFF1F07B501A8FFF7F2FF044A0548B6
:10B620000021121A00F0C0FAF8F7ECF8FEE7C04665
:10B63000086BFF1F1044FF1F01B40248844601BC81
:10B64000604700BF350E000001B40248844601BCCB
:10B65000604700BFDD66010001B40248844601BCBA
:10B66000604700BFE548000001B40248844601BCC1
:10B67000604700BF291C000001B40248844601BC99
:10B68000604700BFE94C010001B40248844601BC98
:10B69000604700BF311B000001B40248844601BC72
:10B6A000604700BF4550000001B40248844601BC19
:10B6B000604700BF014C010001B40248844601BC50
:10B6C000604700BF434D010001B40248844601BCFD
:10B6D000604700BF4551010001B40248844601BCE7
:10B6E000604700BF154D010001B40248844601BC0B
:10B6F000604700BFED3AFF1F01B40248844601BC19
:10B70000604700BF4D1F000001B40248844601BCE1
:10B71000604700BF851F000001B40248844601BC99
:10B72000604700BF0519FF1F01B40248844601BCF1
:10B73000604700BF3D4B010001B40248844601BC94
:10B74000604700BFB14E000001B40248844601BC0E
:10B75000604700BF8B52010001B40248844601BC1F
:10B76000604700BF1D4B010001B40248844601BC84
:10B77000604700BFB139FF1F01B40248844601BCD5
:10B78000604700BF6D36FF1F01B40248844601BC0C
:10B79000604700BFE117000001B40248844601BCC5
:10B7A000604700BF156B010001B40248844601BC2C
:10B7B000604700BF2526000001B40248844601BC52
:10B7C000604700BFB54C010001B40248844601BC8B
:10B7D000604700BFF94C010001B40248844601BC37
:10B7E000604700BF6571010001B40248844601BC96
:10B7F000604700BF017F000001B40248844601BCDD
:10B80000604700BFADAE000001B40248844601BCF1
:10B81000604700BF3119FF1F01B40248844601BCD4
:10B82000604700BFD949010001B40248844601BC09
:10B83000604700BFE538FF1F01B40248844601BCE1
:10B84000604700BF1147010001B40248844601BCB3
:10B85000604700BF5522000001B40248844601BC85
:10B86000604700BFC9A9000001B40248844601BC7A
:10B87000604700BF0D52010001B40248844601BC7C
:10B88000604700BF8D12000001B40248844601BC2D
:10B89000604700BFD91B000001B40248844601BCC8
:10B8A000604700BF5952010001B40248844601BC00
:10B8B000604700BF8530FF1F01B40248844601BCC9
:10B8C000604700BF2146010001B40248844601BC24
:10B8D000604700BF0D31FF1F01B40248844601BC20
:10B8E000604700BF090E000001B40248844601BC55
:10B8F000604700BF0534FF1F01B40248844601BC05
:10B90000604700BF5147010001B40248844601BCB2
:10B91000604700BFC56D010001B40248844601BC08
:10B92000604700BF091B000001B40248844601BC07
:10B93000604700BFC521000001B40248844601BC35
:10B94000604700BFF137FF1F01B40248844601BCC5
:10B95000604700BF056A000001B40248844601BC8C
:10B96000604700BFF938FF1F01B40248844601BC9C
:10B97000604700BF313BFF1F01B40248844601BC51
:10B98000604700BF75A9000001B40248844601BCAD
:10B99000604700BFC926000001B40248844601BCCC
:10B9A000604700BF7918000001B40248844601BC1A
:10B9B000604700BFEDA5000001B40248844601BC09
:10B9C000604700BFC51D000001B40248844601BCA9
:10B9D000604700BF093BFF1F01B40248844601BC19
:10B9E000604700BFE928000001B40248844601BC5A
:10B9F000604700BF4936FF1F01B40248844601BCBE
:10BA0000604700BF1D3AFF1F01B40248844601BCD5
:10BA1000604700BFDD52010001B40248844601BC0A
:10BA2000604700BF055E000001B40248844601BCC7
:10BA3000604700BF3139FF1F01B40248844601BC92
:10BA4000604700BF3D18000001B40248844601BCB5
:10BA5000604700BF3555000001B40248844601BC70
:10BA6000604700BF2951010001B40248844601BC6F
:10BA7000604700BFED4A010001B40248844601BCA2
:10BA8000604700BFC94A010001B40248844601BCB6
:10BA9000604700BFF54E010001B40248844601BC76
:10BAA000604700BF3D36FF1F01B40248844601BC19
:10BAB000604700BF8552010001B40248844601BCC2
:10BAC000604700BFA54F010001B40248844601BC95
:10BAD000604700BFA946010001B40248844601BC8A
:10BAE000604700BF5125000001B40248844601BCF4
:10BAF000604700BF9DA9000001B40248844601BC14
:10BB0000604700BF810E000001B40248844601BCBA
:10BB1000604700BF456B010001B40248844601BC88
:10BB2000604700BF2D2EFF1F01B40248844601BCB0
:10BB3000604700BF3D37FF1F01B40248844601BC87
:10BB4000604700BF6D30FF1F01B40248844601BC4E
:10BB5000604700BF7139FF1F01B40248844601BC31
:10BB6000604700BF350E000001B40248844601BCA6
:10BB7000604700BFD532FF1F01B40248844601BCB4
:10BB8000604700BFCD4C010001B40248844601BCAF
:10BB9000604700BF0124000001B40248844601BC94
:10BBA000604700BF993AFF1F01B40248844601BCB8
:10BBB000604700BFB70E000001B40248844601BCD4
:10BBC000604700BF6DBC000001B40248844601BC60
:10BBD000604700BF2124000001B40248844601BC34
:10BBE000604700BFC53AFF1F01B40248844601BC4C
:10BBF000604700BF5D17000001B40248844601BCE5
:10BC0000604700BF1D3BFF1F01B40248844601BCD2
:10BC1000604700BF691F000001B40248844601BCB0
:10BC2000604700BF1D4D010001B40248844601BCBD
:10BC3000604700BF5549010001B40248844601BC79
:10BC4000604700BFB352010001B40248844601BC02
:10BC5000604700BFF30E000001B40248844601BCF7
:10BC6000604700BF090E000001B40248844601BCD1
:10BC7000604700BFAD32FF1F01B40248844601BCDB
:10BC8000604700BF8D1BFF1F01B40248844601BC02
:08BC9000604700BF594F01009D
:10BC9800000101030202030304030502060207026E
:10BCA800080209030A030B030C020D000E030F031D
:10BCB800100311031303140315001600BD3B0011F4
:10BCC800F13B00110000000002000000DABC001186
:10BCD800192A0F180A000000F1590000FD2400007D
:10BCE8004146010091800011A5A00011F9740011CE
:10BCF800957E00114953001199AE0011954F00111E
:10BD0800CD3D0011FD3E0011000000001616000098
:10BD18000200000024BD0011F4FFF3FFD2FC000074
:10BD28003D400011000000000000000054757961DA
:10BD38000042312E3900303031350067697468753A
:10BD4800622E636F6D2F7076767800544830350018
:10BD5800020000006CBD0011292A282A272A262A59
:10BD6800252A242A0A180000E204000071020000B3
:10BD780078EC000005000000744000001027000067
:10BD880060F000000400000006640000204E00007F
:10BD98000000000006000000050000001F501D0004
:10BDA800023CB4000001150019000000A1020000C7
:10BDB80030313233343536373839414243444546D9
:10BDC800000000004D570011A157001100000000AD
:10BDD80002000000E4BD00116F2A6E2A1A18EAD882
:10BDE800BC80F0FC60000000000000000000F303CD
:10BDF800B59747D6F613F7D777E6F0A7F47400009F
:10BE080001A00000000000006410B71DC8206E3BB0
:10BE1800AC30D9269041DC76F4516B6B5861B24D49
:10BE28003C7105502083B8ED44930FF0E8A3D6D6B3
:10BE38008CB361CBB0C2649BD4D2D38678E20AA01B
:10BE48001CF2BDBDFB349B5F800000800010000029
:10BE580000000000FB600011857700111F610011D0
:10BE68008D7B0011A3610011637B00111962001121
:10BE7800397B00116B620011017D0011D362001142
:10BE8800017D001105630011BB7C001119620011CE
:10BE9800F17A001191620011997C001100000000F4
:10BEA8000000000077630011997C0011D96300112C
:10BEB8009D770011052A042A012A002A022903284D
:10BEC80001280028011800180000000000000000E8
:10BED80000000000000000870101020102010102C8
:10BEE800010203030401030101010101030302012B
:10BEF80003000D000E0010001100130014010701CB
:10BF080008010A010B011C011D02040205020702B7
:10BF1800080219021A021C021D030103020317007A
:10BF28000201000504000807000B0A001716001D8F
:10BF38001C010201010504010E0D01111001141369
:10BF4800011716011A19020201020B0A020E0D024C
:10BF58001110021413021716030504030807030B34
:10BF68000A030E0D0001020307090A0B0E0F101138
:10BF780012141718191A1B1F20212200E1A70011FB
:10BF88009DA800110000000002000000CEBE0011B4
:10BF980000000000C9B50011000000000200000008
:04BFA800CCBE0011FA
:020000041FFFDC
:1000000000000000353D0011E0BC0011DCBC001117
:100010004061FF1F00000000000000000000000021
:1000200000000000000000000000000000000000D0
:1000300000000000000000000000000000000000C0
:1000400000000000000000000000000000000000B0
:1000500000000000000000000000000000000000A0
:100060000000000000000000000000000000000090
:100070000000000000000000000000000000000080
:100080000000000000000000000000000000000070
:100090000000000000000000000000000000000060
:1000A0000000000000000000000000000000000050
:1000B0000000000000000000000000000000000040
:1000C0000000000000000000000000000000000030
:1000D0000000000000000000000000000000000020
:1000E0000000000000000000000000000000000010
:1000F0000000000000000000000000000000000000
:1001000000000000000000000000000000000000EF
:1001100000000000000000000000000000000000DF
:1001200000000000000000000000000000000000CF
:1001300000000000000000000000000000000000BF
:1001400000000000000000000000000000000000AF
:10015000000000000000000000000000000000009F
:10016000000000000000000000000000000000008F
:10017000000000000000000000000000000000007F
:10018000000000000000000000000000000000006F
:10019000F932FF1F5931FF1FC16601000000000046
:1001A000000000000000000000000000000000004F
:1001B000000000000000000000000000000000003F
:1001C000000000000000000000000000000000002F
:1001D000000000000000000000000000000000001F
:1001E000000000000000000000000000000000000F
:1001F00000000000000000000000000000000000FF
:1002000000000000000000000000000000000000EE
:1002100000000000000000000000000000000000DE
:1002200000000000000000000000000000000000CE
:1002300000000000000000000000000000000000BE
:1002400000000000000000000000000000000000AE
:10025000000000000000000000000000000000009E
:10026000000000000000000000000000000000008E
:10027000000000000000000000000000000000007E
:10028000000000000000000000000000000000006E
:10029000000000000000000000000000000000005E
:1002A000000000000000000000000000000000004E
:1002B000000000000000000000000000000000003E
:1002C000000000000000000000000000000000002E
:1002D000000000000000000000000000000000001E
:1002E000000000000000000000000000000000000E
:1002F00000000000000000000000000000000000FE
:1003000000000000000000000000000000000000ED
:1003100000000000000000000000000000000000DD
:1003200000000000000000000000000000000000CD
:1003300000000000000000000000000000000000BD
:1003400000000000000000000000000000000000AD
:10035000000000000000000000000000000000009D
:10036000000000000000000000000000000000008D
:1003700015B60011000000000000000000000000A1
:10038000000000000000000000000000000000006D
:10039000000000000000000000000000000000005D
:1003A0000000000000000000000000000D1BFF1F07
:1003B000000000000000000000000000000000003D
:1003C000000000000000000000000000000000002D
:1003D000000000000000000000000000000000001D
:1003E000000000000000000000000000000000000D
:1003F00000000000000000000000000000000000FD
:08183800106FFF1F4118FF1F94
:10184000024981F3088802F09FFB0000106FFF1F20
:1018500070B500241E491F4A1F484C6308CA1B0567
:101860001B0DE4188242F9D11C4B80228B630021AE
:1018700009201B4B920519621A4B1B4DDA671B4B53
:10188000DA688243DA609A68194802409A60112047
:10189000296002F08DF8112002F06AF880226B6C4A
:1018A000112093436B64EE23DB006343114A1B0C4E
:1018B00013840122104B9A7201F004FC0F4B1B7829
:1018C000002B04D10E4B1021187802F0C5F970BD21
:1018D000000005408805054000060540FF010000A6
:1018E00000F0004004E100E0003800403CF000401F
:1018F000FFDFFFFF1061FF1FC461FF1FF263FF1FC7
:10190000F061FF1F10B502F017FB072804D0122862
:1019100008D0022808D010BD044A0420136B0133FC
:101920001363F8E70220F6E71420F4E7F064FF1FE2
:10193000F8B507000C0026002500503630785135E8
:10194000002804D10300287058342370F8BD29788A
:10195000CA00481E8141A3183800A25C5B68C9B266
:10196000FFF7D0FF00280DD12B78DA00A218013341
:1019700050602B703378044A013B3370136A013393
:101980001362D8E70123DFE7F064FF1F5C234343C2
:10199000074910B5C9180B0058331B78012B05D126
:1019A000FFF7C6FF034A936A0133936210BDC04636
:1019B0002465FF1FF064FF1F10B502F0F5FA064A18
:1019C0000121130010CB4942D967044B136002F088
:1019D000B3F9200010BDC04600E100E01000100087
:1019E00010B5040002F0E0FA024B1C6002F0A4F90A
:1019F00010BDC04600E100E0431E5A425341A02200
:101A0000F0B5D2015B421340154D164A40019B18B8
:101A10002A18127E8BB00191002A1BD01A000832BE
:101A2000D46F0022E6B206AFE4B294420EDC28186E
:101A3000C369002B08D0019902AA117106AA049269
:101A400002AA167303A898470BB0F0BD1978B954D1
:101A50000132EAE71A7D1A7806AB01261A70E6E72A
:101A6000B067FF1F00400040F0B5254B0400400167
:101A7000C25C85B0002A2BD01A18117E002927D00D
:101A8000917E002924D01179022921D11689D78885
:101A9000D168F51BADB22A1C102D00D9102292B2CC
:101AA000BE4217D11818012303710023C269C380F5
:101AB00003819A4206D068460321037301710293A1
:101AC00001A890470820002C00D0192001F0FAFA54
:101AD00005B0F0BD013C65426C41A0256442ED01BA
:101AE0002C40084D1B186419074D0633013A92B279
:101AF000AA42EDD01888461C1E80085C2070F5E7CD
:101B0000B067FF1F00400040FFFF00000F220E4B98
:101B100010B59868104002380A280BD801F0FEFF73
:101B20000D0A0B0A0A110A0A0A0A060002210020FD
:101B3000FFF762FF10BD0121F9E70020FFF794FFD6
:101B4000F8E7DB6FF6E7C046004000400F220E4B7F
:101B500010B59868104002380A280BD801F0DEFF53
:101B60000E0A0B0A0A120A0A0A0A060002210120BA
:101B7000FFF742FF10BD01210800F9E70120FFF740
:101B800073FFF7E7DB6FF5E70090004013B5334CC8
:101B90002378072B3DD8324B1A78324B002A39D1A3
:101BA0008022196852020A431A60252001F0C0FE03
:101BB00020232D4A11680B43802113606B460422B9
:101BC000C90508680733104228D080210422C905BE
:101BD000C86810422ED080212020C905CA688243DF
:101BE000CA6014221A701A78002A2FD18021C905E0
:101BF000C86820320243CA6014221A701A78002A78
:101C000028D11A4B1A7D22785A601D221A70593237
:101C1000DA6013BD1A6816490A40C5E7086802432E
:101C20000A6014221A701A78002ACED01A78013A63
:101C3000D2B2F7E7C8680243CA6014221A70197852
:101C40004A1ED2B21A700029F9D1C4E71A78013AB3
:101C5000D2B2C7E71A78013AD2B2CEE74843FF1FA3
:101C60001044FF1F3CF000404043FF1F0020004095
:101C7000FFFFFEFF564B70B51B68012B03D1554A81
:101C8000936D0133936501F0F7FF534B534A18608E
:101C9000534B544C1A600123534A1360534A136048
:101CA0002378002B06D006225149524802F00CF945
:101CB00000232370504A514B10681B78C1B2002B8F
:101CC0000ED14F4CC0B223785BB2002B4FDB237890
:101CD00024785BB264B21B0424021B191B18136026
:101CE0000B1C50294ED95023464A47491078DBB285
:101CF000FF2202284BD10868444C454D267890437A
:101D00002A78964254D9227824782E78023B5D10A6
:101D1000A31B6B435201D31A10335B1118430860A5
:101D200001F0DAFF031F012B45D83A4B1B78002B3B
:101D300006D0394B1B78002B02D0002002F0BCF8F3
:101D4000A122364B92009978354B4A431B689B1869
:101D5000832292009B181B78033B012B03D8AF20F2
:101D6000400002F089F801222E4BDA8270BD237800
:101D700024785BB264B2FF33FF341B0424021B19C6
:101D80000138ABE7CAB2022AAED20223ACE7086838
:101D9000254C264D267890432A78964208D92278F9
:101DA00024782D78023B5B10641B63435201B2E739
:101DB0002378DBB2B2E70228D5D11D4B1B78013B5B
:101DC000022B03D91B4B1B78022BCCD16C20C8E70C
:101DD0009809FF1FFC0FFF1F3C64FF1FFF3F00001F
:101DE000141003404064FF1F0C1003400010034018
:101DF000D50BFF1F7211FF1FB40003408C09FF1F9A
:101E0000680AFF1F490AFF1F94000340460AFF1F8C
:101E1000470AFF1FF908FF1F2209FF1F300DFF1F90
:101E20003409FF1FBC0BFF1F440AFF1F450AFF1F99
:101E30001C09FF1F2309FF1F10B501F0FDFE002242
:101E4000014B1A8010BDC0463864FF1F10B501F069
:101E500053FFA121054A89009478054A614312681D
:101E6000044B5218528C1A8010BDC046300DFF1F13
:101E70003409FF1F3864FF1F10B50D4B0D4A9978C8
:101E8000A1239B004B431268D218531DD97F0A4BE4
:101E90001B88994209D2441C07D0C82805D0D269B2
:101EA0005B1A5A43054B5343C01802F095F810BD16
:101EB000300DFF1F3409FF1F3864FF1F710200003F
:101EC00070B5244D2B68002B28D001F075FF2B68CE
:101ED000D8402B680400002B27D001F03DFE2B6872
:101EE000D8401D4B1D4A9978A1239B004B43126893
:101EF000D118D25C91239B00002A20D0CA5801320D
:101F0000CA50174B17491B680868834214D3D23B49
:101F1000181A012A1AD0144B186070BD01F04CFF3A
:101F2000124B196801F058FED3E701F015FE0F4B74
:101F3000196801F051FED4E70D495B18E8E7CA5073
:101F40000C4B1B68DB68E418201AE4E7F530FF301F
:101F5000E1E7C0461C08FF1F300DFF1F3409FF1FBB
:101F60009C09FF1F3C64FF1FA009FF1F1808FF1FEB
:101F70002DFF3F004464FF1F70B504000D002829A9
:101F800016D10300A433C2881B889B1A0B4A9BB24C
:101F900093420DD906006A3605223100653001F002
:101FA00023FE002804D13100200002F025F870BD86
:101FB0002900200001F070FEF9E7C046FE7F000016
:101FC000F8B50500012001F047FF134CA36AA26A8F
:101FD0009342FBD1114E336001F0BEFE1049030065
:101FE00008601048426894460F4A17680022BC45B2
:101FF00001D24268BA1A0D4802603268AD18A422B4
:10200000E562606A520302436262094A1278002A5A
:1020100001D00F3B0B60F8BD00F00040340AFF1FF9
:10202000E408FF1F28100040180AFF1F1C0AFF1FAA
:102030001C09FF1F70B580241025E405A3682B43FD
:10204000A36001F0A1FEA368AB43A36070BD0000D4
:10205000F7B5160080221C001023D205019191686B
:1020600005000B43936000225A4BD7301A6001F0F1
:1020700053FE9D232A002F009B00EB58CA320121FA
:102080000092FC37002B01D00021009A386801F043
:1020900013FE2900009BCB311A784F4BD3351A60C1
:1020A0004B780A781B0213438A7812041A43CB78C0
:1020B0001B061343494A1BBA13604B790A791B026A
:1020C00013438A7912041A43CB7931001B06134358
:1020D000434A1BBA13606B782A781B021343AA7811
:1020E00012041A43EB781B0613433E4A1BBA1360D3
:1020F000019A330213433C4A13603C4B22001B1BE2
:102100009C4603293DDCB3089A0013005142B21AE1
:10211000032A46D1354AE018511A827840781204D1
:1021200000020243E05C043302430A600022FF2BFA
:102130004BDDF0222E4B12011A600F222D4B1A603C
:102140002D4A1368002BFCD00023224A2749136034
:10215000091B321D0B191B68043A180A23706070A2
:10216000180C1B0EA070E3700434002AF2DC8022ED
:1021700010213B68D20501333B6093688B43936029
:10218000F7BD6346D578981893782D061B042B432A
:10219000157804392B43557804322D022B43036004
:1021A000AFE7022A0AD1114AE05C511AE2185278CC
:1021B000120202430A6004339BB2B7E7012AB5D189
:1021C0000A4A521AE15C1160F5E7084959180A6099
:1021D0000433ACE7000004403C00044038000440F5
:1021E00034000440300004400C000440000104406E
:1021F000040004401000044014000440F7B515002A
:1022000080221C001023D2050091916807000B4327
:1022100093600023654AD730136001F07DFD9D2354
:102220003E009B00F9583B00CA363200FC330029BF
:1022300000D07FE0586801F03FFD390032785C4BF8
:10224000CB311A604B780A781B0213438A78AC466C
:1022500012041A43CB78281D1B061343554A1BBA98
:1022600013604B790A791B0213438A7912041A43CB
:10227000CB791B061343504A1BBA13604B7A0A7A78
:102280001B0213438A7A12041A43CB7A21001B06DD
:1022900013434A4A1BBA1360009A2B021343484A5D
:1022A00013602200474B1B1B0093009BCE785B18EA
:1022B00001938B7836061B0433430E78043833437E
:1022C0004E78043136023343019E33600328ECDC40
:1022D0000321A808431C9B002940800003292BD11F
:1022E0003849E5185E18A9786D78E35C09042D0279
:1022F000294319433160030008330021FF2B2DDDF2
:10230000314B324919600F21314B196001232749A4
:102310000B60304B19680029FCD006211B680B406C
:10232000042B20D080220020D20593680A318B43F1
:102330009360FEBD01217DE7022908D121495D1886
:10234000E1184978E35C090219432960D3E70129C0
:10235000D3D11C495918E35C0B60CCE71948181815
:1023600001600433CAE7002310490B606346002B69
:102370000CDC3B00FC335A68102101325A60802289
:10238000D205936801208B439360D2E7009B9B1892
:102390001B68190A13705170190C1B0ED37004239B
:1023A0005B4291709C440432E0E7C0460000044068
:1023B0003C00044038000440340004403000044035
:1023C0000C0004400001044004000440080F000019
:1023D000100004401400044070B5061E19D00222FB
:1023E0005A4B9B799343012B13D1594B1A78FF2AEF
:1023F0000FD15A78FF2A0CD19A78FF2A09D1DA78BE
:10240000FF2A06D11A79FF2A03D15B79FF2B00D16D
:1024100099E0504B0C201A78012A08D000224E4D2A
:102420001A7029780B00093B042B01D8212070BDBC
:102430004B1F012BFAD9454CA37B042B00D982E01A
:10244000A279032A00D97EE09A1ED2B2012A02D8CC
:1024500060881F2877D9002E56D0012E73D1A0880E
:102460000128E3D0002907D1581E032803D801F022
:1024700055FB121715122E702978481E032811D803
:102480000025364B1D602823237501F00DFDA84261
:1024900027D0A580CAE702212970EDE70421FBE7D8
:1024A0000321F9E707390129C0D82D490968C96A0C
:1024B0008906BBD52B4908780028B7D1012A01D954
:1024C000002BB3D102230B708021274D26338901C5
:1024D0002878237501F090FB80212878890101F08C
:1024E000BBFB0123A380214B1B78002B0AD0FA22CF
:1024F00080211F4B92001B8809025A431A4B1878FF
:1025000001F012FC002092E701F04EFD2B78A6802E
:10251000073B012B03D917482E7001F0B5FC114B76
:10252000114C1A78002A06D08021002220788901D7
:102530001A7001F061FB01F0FFFB80212078090295
:1025400001F05AFBDEE7122071E7C046A60BFF1F21
:102550006B09FF1F1A09FF1F1C09FF1F4809FF1FF6
:102560004464FF1F2309FF1F1B09FF1F2109FF1FD1
:102570002C09FF1F0010004010B5002901D001F008
:1025800043FB10BDF7B5604B01919978A1239B00E7
:102590004B435E4A060014681022E418D6235B0001
:1025A000E0583623FF33E35C00279343222B41D1CD
:1025B000574B0F3A1A600760012501F0A5FC019BFB
:1025C0001880E8235B00E35C002B01D0B34258DDA8
:1025D0000023504FFB70AD33FF33E3581A68002AD5
:1025E00003D09B88DB439B071DD03823FF33E35C7C
:1025F000002B18D09B235B00E35C002B13D1D1335D
:10260000FF33E35CB3420EDAA4235B00E15AE01827
:10261000090A023101F028FC23000122FE33013EA9
:1026200001351A87FA70E8235B00E35C002B2AD09F
:10263000A8B2FEBD03683D00002BBED081880430E7
:10264000090A023101F010FCD6235B00E3581F6039
:10265000B2E72300B133BA00FF33985801378188BD
:102660000430090A023101F0FFFBE8235B00E35C60
:10267000BB42EEDCE822F61AED1800235200A35408
:10268000A6E70027F1E7200001F00EFB00281FD08D
:10269000002E1DDD7319882647190193B60020000E
:1026A00001F07AFC5A30800020184068013581889A
:1026B0000430090A023101F0D7FB200001F00CFCC4
:1026C000A3590133A351BD4202D0019B9D42E6D1E3
:1026D000114BE35C002BABD095239B00E35C002BFC
:1026E000A6D00E4BE15A0029A2D00D4AA35C994214
:1026F00002D90133A3549BE700231A212000A354DD
:1027000001F012FC94E7C046300DFF1F3409FF1F93
:1027100000140340E010FF1F5A0200007202000084
:102720005E0200000D4970B54A6E0D4CD2038B69F4
:10273000D20BA24206D80B4D0224AA4204D901F0C2
:1027400053FB70BD02246442E21815007E2425402C
:102750002242F4D0A3432B438B61F0E700F000400A
:102760000A200000FC1C0000F8B51D4B1D4F1A7814
:10277000002A10D1BA7B002A02D101321A7003E07C
:10278000032AFAD0022AF8D001F08EFB00220120A1
:10279000154B1A70F8BD154B154D1C68154B9E78DE
:1027A00001232B702878C0B200F09EFBBB7B002B6E
:1027B0000BD101F0C9FAA1239B007343E4188323D2
:1027C0009B00E41823782B70E4E7032B02D101F07F
:1027D0002BFBF0E70020022BDCD101F025FCEAE71F
:1027E0001C09FF1FA60BFF1F2309FF1F3409FF1F32
:1027F000490AFF1F300DFF1FF0B587B00EAD2F78CF
:102800000FAD2D780593AC46634614000E4D0CAA0F
:1028100012782E7803930D9B009201932200059B62
:10282000029701F0D1FA2E70012C01D0042C08D1AE
:10283000802206498B889343054A1278D2011343BC
:102840008B8007B0F0BDC0461C09FF1F6C11FF1F35
:102850007809FF1F0B001B3B70B504003020E02BF4
:102860000DD81300E025493BFF3B9BB2ED00AB4286
:1028700005D8034B200019825A8201F0E5F970BD9A
:102880008410FF1F10B501F0F7F9054B00205B68BD
:10289000052B04D9034A5268D20200D4980810BD0F
:1028A00000100040FCE100E070B501F07DFB0D4B35
:1028B0001B68FC33DC691D6AFFF7E4FF641984427E
:1028C00004D2094B01241B68002B07D004220024EA
:1028D000064B1A70064A93690133936101F02CFA92
:1028E000200070BD4464FF1F9809FF1F2309FF1FCC
:1028F000FC0FFF1F70B50C4D2B68FC335C6A01F0B8
:1029000053FBFFF7BFFF2B680025FC339B6AE318DE
:10291000834204D2054B1B68AB4200D1051B01F07A
:102920000BFA280070BDC0464464FF1F9809FF1FC2
:10293000D722044B92009B5810B5002B00D098472B
:1029400010BDC0460000FF1F10B501F0CFF8FFF723
:10295000EFFF2749274BCA6D274C1A4084235B00A1
:102960001343CB65254B1B68186A01F075FA244B9D
:10297000244A1A60244B254A1A60A022244B520094
:102980001A60244B187801F03FFA2000224901F028
:10299000DBFA0023A3600233A360204B20492360AD
:1029A00003232048A36001F0CFFA10221E4BFF2022
:1029B0001A60802252031A60802292031A608022D9
:1029C00012041A6001F078FA012001F0CDFAFA2021
:1029D000400001F0F9FA582001F04EFA134801F0D6
:1029E000FBF9012001F0B8FA072001F07DFA10BDD3
:1029F00000F0004000FEFEFF141000404464FF1F82
:102A0000000003400180063DBC0003403408000084
:102A1000A40003404A0AFF1F71020000C30900001E
:102A2000FFFF3F002810004000E100E0307500008B
:102A3000674E336888331B6883F3088801F0E4FA33
:102A4000644A6549136800200B401360634B644A75
:102A50001B68934200D1A6E001F0C6FA0221614A48
:102A600013688B431360FFF76FFF5F4B5F4C187861
:102A7000C0B201F091F80023A3600233A3605C4B65
:102A80000120236001F0E8F90323A36001F0CCF8F2
:102A9000040001F0F1F8050001F0C6F8554B18608C
:102AA00001F082F9544B1968621A531EA14200D2F8
:102AB00013008022D203934201D39B029B0A326807
:102AC000D16AC90700D471E04C491C0C09689BB25B
:102AD0004C4359432402090A641803264849FC322E
:102AE00093680A6847489B1A474A0768126847492B
:102AF0009B18474A9A1833409208DB190A60036012
:102B0000042B03D9013233400A6003600E68414947
:102B1000A619300001F060F83F4F3E493B68C318EA
:102B20003B603000019301F087FA3C4E3068081892
:102B300038493060884205D9019B01333B6001F080
:102B40007BFA316001F018F9354B1B78002B0DD062
:102B500001F092F8334B621B196812188A4232D284
:102B60004919091B091A304801F0EEF92F4E337A42
:102B7000002B0ED001F080F8621BF1681218914210
:102B800024D94919091B091A294801F0DDF9002344
:102B90003372284B83F3088800F0E6FF002001F031
:102BA00023FA01F071F801F01FFA5CE7DC019900EB
:102BB0000234641A5900641A09214B438033CB4014
:102BC000A408E41889E7FA218900CCE71A49DBE771
:102BD0004464FF1F1CF00040FFFFC1FF0C0AFF1FF1
:102BE000B641210310000040490AFF1F14100040A5
:102BF000C3090000100AFF1F340AFF1F380AFF1F15
:102C0000200AFF1F280AFF1F1C0AFF1F240AFF1F9C
:102C1000C4090000710200006008FF1F2C0AFF1F9A
:102C20001C09FF1FE408FF1F00100040740BFF1F6A
:102C30003C10004000000020DC050000A022054BF5
:102C400092009B5810B5002B01D0984710BD01F0A1
:102C500023F9FBE70000FF1FA122054B92009B58C0
:102C600010B5002B01D0984710BD01F015F9FBE716
:102C70000000FF1FA222054B92009B5810B5002BAD
:102C800001D0984710BD01F007F9FBE70000FF1FD6
:102C9000A322054B92009B5810B5002B01D09847FA
:102CA00010BD01F0F9F8FBE70000FF1FA422054B5F
:102CB00092009B5810B5002B01D0984710BD01F031
:102CC000EBF8FBE70000FF1F70B500F0D5FF4F4B9E
:102CD000186000F079FF0400C30702D400F064FF1D
:102CE00070BD00224A4B1A604A4B187801380428FC
:102CF00029D800F013FF0320181C2400200000F046
:102D0000B3FF0128ECD0444C2378042B6ED100F0A3
:102D100053FF0028E4D000F07FFF582001F0ACF80A
:102D200002232370DCE7200001F076F9E9E72000B8
:102D300001F062F8E5E7200001F03EF9E1E720004C
:102D400001F01AF9DDE700F0C7FF0500012808D1FE
:102D5000324B1B78053B012B03D82000FFF76EFF99
:102D6000D1E72D4B1B78022B01D0052B20D1022D52
:102D700028D12B4B9B7BAB431CD12000FFF76CFF72
:102D8000264B18780128BED16405BCD424492522DD
:102D90004B7B034205D1233A13405A425341263319
:102DA0001A000B7D9342AED9322000F0DDFFAAE776
:102DB000022D07D1194B1B78052B11D12000FFF7ED
:102DC00059FFDDE7012D0BD1012B03D12000FFF7C7
:102DD0005FFF98E7062B03D12000FFF767FF92E71C
:102DE000200001F059F8022D8DD1C9E7032B04D141
:102DF0000C4B987C00F088FF72E7072B00D06FE740
:102E0000094B987B00F0B8FE6AE7C0469C09FF1F9B
:102E10009809FF1F9009FF1F2309FF1F1C09FF1FAF
:102E2000A60BFF1FBC0BFF1FD40BFF1FFA210A4B81
:102E30000A4A49001A640A4A5A500A4A04395A503E
:102E4000094A08319A64094A5A50094A5C315A5071
:102E5000084ADA667047C0460000FF1FF927FF1FC7
:102E6000F528FF1FA928FF1FD923FF1F6927FF1F70
:102E7000791EFF1F4D1EFF1FF7B50B0CFF27012208
:102E8000009300233C001E001D009446019089B26F
:102E900062469A401000084018413618B6B2FF2F1B
:102EA00002D1012E00D19FB2009802401A41AD1804
:102EB000ADB2FF2C02D1012D00D19CB20133102BF9
:102EC000E6D10320012E07D1012D04D1019B24015D
:102ED000E4191C700138FEBD102EFCD10238102DF3
:102EE000F9D00230F7E700008023F7B59C46264B67
:102EF000264F01932649274A274D284C284B022864
:102F00001AD1604638600868264E30408026360365
:102F10003043086001990978002909D11660224AD6
:102F20002A60224A2260E02219689143A03A1BE0FD
:102F30008021C9021160F2E766463E600F68194EB3
:102F40003E408027FF023E430E6001990978002928
:102F50000DD1176001280ED1154A2A60154A22604A
:102F6000E02219689143C03A0A431A60F7BD8021F4
:102F700089021160EEE7E0210F4A02432A600F4AFE
:102F800022601A688A43F0E74B0AFF1FE000034003
:102F9000D80003409000034000000340500003406D
:102FA00040000340FFFFE3FF0280063D804508220A
:102FB0000180063D80660822008006988055082220
:102FC000F8B51E4B80261A680020140034403242A7
:102FD00032D11A681A4F32431A6001223B68063018
:102FE00093433B6000F038FF0122164D2B681E43CF
:102FF0002E603B680A2613433B608027BF00124BBC
:103000001B683B4211D1013EF6B2FF2E09D17E2250
:103010000E4B1C682B68E40B1440934323432B6036
:1030200005E0082000F018FFE9E7002EEFD180222C
:103030002B68600893432B60F8BDC046C4F0004085
:103040005CF0004018F0004068F0004060F0004084
:1030500010B500F061FF01215820034A00F044FE42
:10306000FFF7AEFF10BDC046600AFF1F10B5782203
:103070000021034800F0D0FE00F066FD002010BDE6
:103080003867FF1F70B5040000F08EFF00230C208E
:103090000B4A010059438D18515C00290DD0A14203
:1030A00008D1012300246B7000F026FF00F044FEDD
:1030B000200070BD01330A2BEBD11224F6E7C04685
:1030C0003867FF1F70B5040000F06EFF0023190081
:1030D0001D000D4A1078002806D0A0420CD1557072
:1030E00001310C320A29F5D1002B0AD100F02CFD58
:1030F00000F022FE002070BD5078461EB0411B1823
:10310000EEE700F0F9FEF3E73867FF1FF7B50400BC
:103110000C20002384460E4D019267465F43E85D14
:103120007E19A04212D000280BD10A4B9C46624661
:103130001B7808331370019B70707C557160B3600D
:10314000FEBD01330A2BE8D10320F9E70720F7E79A
:103150003867FF1F3467FF1F8020F8B5484BC00554
:103160001B68C1248360474BFF251A680123134362
:103170004361454BA4001A68444B40211A60444BFC
:103180001A68444B1A60444B1A59AA431A51C52273
:1031900092009E58AE433143802699509F583F4934
:1031A000F6010F403E439E509E5880273602360A55
:1031B0003043985080201A5900020A4002431A51A5
:1031C00004341A59364E3F04324080263A431A518D
:1031D0001A5936061202120A32431A5108341A5981
:1031E00080260A4002431A51C32292009F58B446D7
:1031F000AF4337439F509F58294E0F4007439F507E
:103200009F58374080263604374380269F509F586A
:1032100036063F023F0A37439F50C0221F59AF4333
:103220003A431A511A591202120A1643C6221E5163
:1032300092009C58AC4365462C439C509C580025FA
:103240000C4020439850C72080001A58154C11405C
:10325000C02212020A431A50134B1B78DB08AB4200
:1032600001DC0020F8BD2378002B06D0A368002BDA
:1032700000D0984701350C34EEE71220F2E7C04643
:103280004443FF1F4043FF1FB0F000403067FF1F63
:10329000B4F000402C67FF1F00E100E0FF00FFFFDB
:1032A000FFFF00FF3867FF1F3467FF1F030010B5E3
:1032B0001F2809D8072200201340072404490A7850
:1032C000A24313430B7010BD00230620F5E7C04650
:1032D0003467FF1F054B06491B780A6805485B07E2
:1032E00002401B0B134300200B6070473467FF1F25
:1032F0001CF00040FFFFC1FF70B50C25FFF7EAFF8F
:103300000A4B1C780A4BE4086543ED18002C01D1E8
:10331000200070BD2B78002B06D06B68002B00D0EE
:103320009847013C0C3DF1E71220F2E73467FF1F9C
:103330002C67FF1F1FB5002102220B000191009195
:10334000052000F021FC02230B490A681A42FCD137
:1033500020230393039B5A1E0392002BFAD1074AA2
:103360001368002BFCDA0B246C442000012100F0D0
:103370006BFD207804B010BD90C8004000C800402C
:1033800013B504000A4B0193019B002B01D11120BE
:1033900016BDFFF7CFFF23000340044205D00520F0
:1033A00000F05AFD019B013BEDE71800F0E7C04635
:1033B000FFFFFF0707B500F0F7FD80220821D205C7
:1033C000936A0191002B01D10739916202210C4AC5
:1033D00011600199481E01900029FAD10331116052
:1033E000053101910199481E01900029FAD111601F
:1033F000002B02D18022D205936200F09DFC07BD14
:1034000000C00040F0B52D4C89B02378002B4FD17F
:10341000FEF7D2FA02232A4F03903A681A42FCD1EF
:1034200020230693069B5A1E0692002BFAD1254EA6
:103430003368002BFCDA0120FFF7A2FF011E02D047
:10344000112009B0F0BD030003220190009005ADEA
:103450009F2000F099FB0321280000F0F5FC0223D7
:103460003A681A42FCD120230793079B5A1E079201
:10347000002BFAD13368002BFCDA0120FFF780FF24
:103480000028DDD10398FEF7ABFAAA786B78110417
:103490001B020B4329780B4363601300113B0A495D
:1034A000052B07D801239340A3600B6001232370F1
:1034B0000020C6E780231B03F6E7C0462C43FF1F0E
:1034C00090C8004000C800409808FF1F1E4B30B550
:1034D0005A6818781D4B85B0D31859424B410121C9
:1034E0000093002300F0F0FB194B1A4A02259A635F
:1034F00000221A6510325A658022C4219D65164B40
:103500001648D202DA6789004258154B80241A40C7
:1035100080231B0413434350642341200393E40599
:1035200000F006FA402000F003FA6562039D6B1E6E
:103530000393002DFAD103236362FFF73BFFA562DB
:10354000FFF760FF05B030BD3843FF1F95FFFEF762
:1035500000C80040050001FF04E100E000E100E0D8
:10356000FFFF00FFF0B585B00700FEF725FA022344
:1035700005002D4C22681A42FCD120230093009BA9
:103580005A1E0092002BFAD1284E3368002BFCDA29
:103590000120FFF7F5FE002803D01124200005B01C
:1035A000F0BD234B2360022322681A42FCD1202362
:1035B0000193019B5A1E0192002BFAD13368002B14
:1035C000FCDA0120FFF7DCFE0028E6D1194B1F6072
:1035D000022322681A42FCD120230293029B5A1E26
:1035E0000292002BFAD13368002BFCDA0120FFF79E
:1035F000C7FE0028D1D1104B2360022322681A4253
:10360000FCD120230393039B5A1E0392002BFAD173
:103610003368002BFCDA0120FFF7B2FE041EBCD198
:103620002800FEF7DDF9B9E790C8004000C8004067
:1036300001000006A8C800400180000110B500206C
:10364000FFF790FF10BD000010B5064B18705960D1
:10365000FFF73CFF00211320034AFFF757FD00202E
:1036600010BDC0463843FF1FCD34FF1FF0B5040026
:1036700085B003920291FEF79FF9882263035B0BEA
:1036800052051A438023DB059D6A8023274F009251
:10369000BA68002601901B039A420CD9F823260031
:1036A0001B041E401C4206D08022214B52025E6247
:1036B00019680A431A60002D0BD100F075FC022234
:1036C0001C4B1A608023DB055A62013A9A6200F0B3
:1036D00033FB0023039A934220D1002D0AD100F03E
:1036E00063FC144B03221D608023DB055A629D623C
:1036F00000F022FB8023BA681B039A4208D9002EEF
:1037000006D000220A4B0C495A621A680A401A6015
:103710000198FEF765F9002005B0F0BD009A029906
:10372000D2181278CA540133D4E7C0462C43FF1F85
:1037300000C8004000C00040FFFFFEFFF0B587B0AA
:10374000029103920400FEF737F9019000F02CFC7F
:10375000802302250122234EDB0535605D629A62DB
:1037600000F0EAFA204F3B682B42FCD1202304935F
:10377000049B5A1E0492002BFAD11C4D2B68002B7F
:10378000FCDA0120FFF7FCFD002802D0112007B071
:10379000F0BD2000039A029900F0FEFA0223040013
:1037A0003A681A42FCD120230593059B5A1E0592C4
:1037B000002BFAD12B68002BFCDA0120FFF7E0FD8B
:1037C000051EE3D100F0F0FB80230322DB0535600A
:1037D0005A629D6200F0B0FA0198FEF701F9E0B27A
:1037E000D5E7C04600C0004090C8004000C8004077
:1037F000F0B5802489B00600FEF7DEF8E405A36A80
:1038000002250393029000F0CFFB0123304F3D606F
:103810006562A36200F090FA2E4C23682B42FCD123
:1038200020230593059B5A1E0592002BFAD12A4DA1
:103830002B68002BFCDA0120FFF7A2FD002803D043
:103840001124200009B0F0BD244B2360022322681C
:103850001A42FCD120230693069B5A1E0692002B87
:10386000FAD12B68002BFCDA0120FFF789FD021E3C
:10387000E6D11B4B03211E60030001900090202025
:1038800000F082F9022322681A42FCD12023079318
:10389000079B5A1E0792002BFAD12B68002BFCDAEB
:1038A0000320FFF76DFD041ECAD100F07DFB8023CD
:1038B0000322DB053C605A629C6200F03DFA039BE8
:1038C000002B01D1FFF776FD0298FEF789F8B8E7E3
:1038D00000C0004090C8004000C800400100000641
:1038E00094C8004007B5000201910422000A01A912
:1038F000FFF724FF0EBD000073B5050005240B4A39
:10390000A3005B429B1819686B46DE1D3000FFF771
:10391000B3FA022804D133782B55013CEFD276BD9F
:10392000052CFCD00128FAD10230F8E71409001167
:103930001F2807D8012380228340D20591680B43BA
:10394000936070473F2808D80123802220388340A5
:10395000D20551690B435361F3E75F28F1D8012386
:10396000802240388340D205116A0B431362E8E796
:103970001F2807D8012280218240C9058B68934304
:103980008B6070473F2808D8012280212038824070
:10399000C9054B6993434B61F3E75F28F1D80122D6
:1039A000802140388240C9050B6A93430B62E8E7E7
:1039B0001F2810D880230200DB05153A1968012A58
:1039C00006D820229143196019680A431A6070478B
:1039D00001228240F6E73F2811D880230200DB0550
:1039E000353AD968032A06D810229143D960D9689C
:1039F0000A43DA60EBE7012220388240F5E75F28CE
:103A0000E5D842238022181A413B8340D205516AEF
:103A100099435162516A0B435362D8E710B50400D1
:103A2000012813D1A022184992050B685B015B099C
:103A300013430B60154B164A19681140154A0A4387
:103A40001A60402219680A431A6010BD0028FCD190
:103A500001000A2000F0F0F921000B2000F0ECF941
:103A6000C0220A4B920019680A4340211A601A6862
:103A70008A431A60B022044912060B685B015B0995
:103A800013430B60E1E7C04614F000401CF0004017
:103A90007F00FEFF80FD010072B6074A1368013304
:103AA00013600422054B1A600023054A136080222C
:103AB000D2055360FEE7C0467808FF1FC0F0004003
:103AC000C4F0004005490B68002B05D1044A0A6088
:103AD00004490A60044A13607047C046140AFF1F75
:103AE000841E0000380AFF1FC4F000400023034A70
:103AF0001360034A1360034A1360704754F0004098
:103B000040F1004044F1004002B4714649084900C8
:103B1000095649008E4402BC7047C04602B4714643
:103B200049084900095C49008E4402BC7047C04600
:103B300003B47146490840004900095A49008E44BF
:103B400003BC70470000000001B40248844601BC79
:103B5000604700BFADAE000001B40248844601BC1E
:103B6000604700BF6D0B010001B40248844601BCF0
:103B7000604700BF7997000001B40248844601BC49
:103B8000604700BFC1F7000001B40248844601BC91
:103B9000604700BF496D010001B40248844601BC82
:103BA000604700BF8914010001B40248844601BC8B
:103BB000604700BFDD0A010001B40248844601BC31
:103BC000604700BF01D7000001B40248844601BC31
:103BD000604700BFBD0B010001B40248844601BC30
:103BE000604700BF090E000001B40248844601BCD2
:103BF000604700BFCD4C010001B40248844601BCBF
:103C0000604700BFB352010001B40248844601BCC2
:103C1000604700BFE9D4000001B40248844601BCFB
:103C2000604700BF6DF6000001B40248844601BC45
:103C3000604700BF156B010001B40248844601BC17
:103C4000604700BF8D82000001B40248844601BC79
:103C5000604700BF116E000001B40248844601BCF9
:103C6000604700BF0D52010001B40248844601BC08
:103C7000604700BF0134010001B40248844601BC22
:103C8000604700BFC95C010001B40248844601BC22
:103C9000604700BF8552010001B40248844601BC60
:103CA000604700BF51B8000001B40248844601BC1F
:103CB000604700BF71B0000001B40248844601BCF7
:103CC000604700BF2144000001B40248844601BCA3
:103CD000604700BFC56D010001B40248844601BCC5
:103CE000604700BFDD0C010001B40248844601BCFE
:103CF000604700BF0167010001B40248844601BC6F
:103D0000604700BFF9ED000001B40248844601BCE1
:103D1000604700BF4DF9000001B40248844601BC71
:103D2000604700BF8944000001B40248844601BCDA
:103D3000604700BF8B52010001B40248844601BCB9
:103D4000604700BF9DA9000001B40248844601BC41
:103D5000604700BFE9F6000001B40248844601BC98
:103D6000604700BFBD5C010001B40248844601BC4D
:103D7000604700BF6137010001B40248844601BCBE
:103D8000604700BFD544010001B40248844601BC2D
:103D9000604700BFDD3F000001B40248844601BC1B
:103DA000604700BF9573010001B40248844601BC1E
:103DB000604700BFC166010001B40248844601BCEF
:103DC000604700BFE90B010001B40248844601BC12
:103DD000604700BF9D6A000001B40248844601BCF0
:103DE000604700BF8D11010001B40248844601BC48
:103DF000604700BFD1AE000001B40248844601BC58
:103E0000604700BF0534010001B40248844601BC8C
:103E1000604700BFEDA5000001B40248844601BC24
:103E2000604700BFB70E000001B40248844601BCE1
:103E3000604700BF75F8000001B40248844601BC29
:103E4000604700BF75A2001101B40248844601BC5E
:103E5000604700BF3D71010001B40248844601BCC7
:103E6000604700BF0189000001B40248844601BCDC
:103E7000604700BFC115010001B40248844601BC7F
:103E8000604700BF7912010001B40248844601BCBA
:103E9000604700BFC1A5000001B40248844601BCD0
:103EA000604700BFE917010001B40248844601BC25
:103EB000604700BFA9D8000001B40248844601BC95
:103EC000604700BFED6B010001B40248844601BCAD
:103ED000604700BFE94C010001B40248844601BCC0
:103EE000604700BF5976010001B40248844601BC16
:103EF000604700BFF90D010001B40248844601BCCF
:103F0000604700BF21A9000001B40248844601BCFB
:103F1000604700BFCD0C010001B40248844601BCDB
:103F2000604700BFED68010001B40248844601BC4F
:103F3000604700BF53B9000001B40248844601BC89
:103F4000604700BFE927000001B40248844601BC75
:103F5000604700BF2D6C010001B40248844601BCDB
:103F6000604700BFE512010001B40248844601BC6D
:103F7000604700BF6911010001B40248844601BCDA
:103F8000604700BFF935010001B40248844601BC16
:103F9000604700BF1DB6001101B40248844601BC51
:103FA000604700BFD9B0000001B40248844601BC9C
:103FB000604700BF75A9000001B40248844601BCF7
:103FC000604700BFF535010001B40248844601BCDA
:103FD000604700BF8512010001B40248844601BC5D
:103FE000604700BF8937010001B40248844601BC24
:103FF000604700BF016C010001B40248844601BC67
:10400000604700BF85C1000001B40248844601BC7E
:10401000604700BFC9A9000001B40248844601BC42
:10402000604700BF0934010001B40248844601BC66
:10403000604700BF19FA000001B40248844601BC81
:08404000604700BF090E0000FB
:1040480002000000CABE001101000000D0BC00112F
:1040580002000000C6BE0011010000008840FF1FDA
:1040680002000000D8BC001101000000C061FF1F61
:1040780002000000C4BE0011030000003461FF1FED
:104088001200000002000000CABE0011010000007A
:1040980018BD001102000000C6BE0011010000009A
:1040A80015BD00110200000022BD00110300000030
:1040B8006F61FF1F02000000C4BE00110300000072
:1040C8008461FF1F02000000C6BE0011010000004D
:1040D80014BD00110200000020BD00110300000003
:1040E8004561FF1F02000000C4BE0011030000006C
:1040F8006661FF1F02000000CABE00110100000037
:1041080058BD001102000000C6BE001101000000E9
:10411800D141FF1F020000006ABD0011010000002C
:1041280053BD001102000000C6BE001101000000CE
:10413800D041FF1F0200000068BD0011010000000F
:104148008C61FF1F02000000C6BE001101000000C4
:10415800CF41FF1F0200000066BD001101000000F2
:1041680043BD001102000000C6BE0011010000009E
:10417800CE41FF1F0200000064BD001101000000D5
:104188003EBD001102000000C6BE00110100000083
:10419800CD41FF1F0200000062BD001101000000B8
:1041A80039BD001102000000C6BE00110100000068
:1041B800CC41FF1F0200000060BD0011010000009B
:1041C80034BD0011020202020202000000000000D9
:1041D80016150000B14B0011774B0011B8BD001146
:1041E80090011D0018001800FFFF070102030405D5
:1041F80006020106000000000000000000000000A8
:1042080000000000000000000000000000000000A6
:104218000300000002000000CABE001101000000F7
:10422800D8BD001102000000C6BE00110100000048
:104238008C42FF1F02000000E2BD001101000000D7
:10424800BA61FF1F02000000C4BE00110300000095
:104258002464FF1F02000000C6BE00110100000018
:104268008C42FF1F02000000E0BD001101000000A9
:10427800BC61FF1F02000000C4BE00110300000063
:104288001C64FF1F12A6A6A6000000000000000084
:10429800161500000001000000000111FFFF0000DA
:1042A8005048593600000000000000000B000500CF
:1042B800F0000000B4000028002800283075A00095
:1042C800A000A000A00000080008E001F000100015
:1042D8001000100010001000100050005000500096
:1042E80010001000D0070000000000000F000100BF
:1042F8000500307507001000010081FF0000000074
:10430800FF0000005D74001165720011F56F001167
:10431800FFFF0100FF000000799E0011F59B0011CE
:104328000D9B0011000000000000000000000800C4
:10433800040000003B0001085902E0018821280020
:10434800FF00000002000000CABE001101000000CA
:1043580090BF001102000000C6BE0011010000005D
:10436800C943FF1F02000000C2BE00110100000087
:10437800F067FF1F02000000C6BE00110100000028
:10438800C843FF1F02000000C0BE0011010000006A
:10439800C643FF1F02000000C6BE00110100000056
:1043A800C443FF1F02000000BEBE00110100000050
:1043B800BC43FF1F180018001D00900102000003F5
:1043C8000202000002000000CABE00110100000045
:1043D800A4BF001102000000C6BE001101000000C9
:1043E8000C44FF1F02000000BCBE001100000000CA
:1043F8000000000002000000C4BE0011030000001D
:064408001068FF1F20FFF9
:040000051FFF184180
:00000001FF
